:020000040800F2
:10500000C01B0020D5500008998C0008718300084F
:105010000000000000000000000000000000000090
:10502000000000000000000000000000D59900080A
:10503000000000000000000079920008ED9A0008CE
:10504000E7500008E7500008E7500008E750000864
:10505000E7500008895D0008E7500008E7500008A5
:1050600000000000E7500008B15C0008E7500008AD
:10507000E75000088988000800000000E750000899
:1050800000000000E75000080000000000000000E1
:10509000E750000800000000E7500008E750000853
:1050A000E7500008E7500008E750000899A50008FD
:1050B000E7500008E7500008000000000000000072
:1050C0000348854600F040FD0048004719B9000834
:1050D000C01B00200448804704480047FEE7FEE765
:1050E000FEE7FEE7FEE7FEE7899B0008C1500008E7
:1050F00030B50B46014600202022012409E00D4670
:10510000D5409D4205D31D469540491B25469540F7
:1051100040191546521E002DF1DC30BDF0B51FB40C
:105120000646002082B005464024019100901BE015
:10513000019922460F46304600F0F0FB049A059B89
:10514000801A994110D310461946224600F0D6FB2A
:10515000361A8F410197224601200021009F00F05E
:10516000CDFB38184D4100902046641E0028DFDC3E
:10517000019B00982946324607B0F0BD03460B4319
:105180009B0703D009E008C9121F08C0042AFAD2FD
:1051900003E00B780370401C491C521EF9D2704783
:1051A000D2B201E00270401C491EFBD270470022BF
:1051B000F6E710B513460A4604461946FFF7F0FF16
:1051C000204610BD30B504460020034600E05B1CBD
:1051D000934203D2E05CCD5C401BF8D030BDF8B503
:1051E00002464A40D40F42004B0052085B089A42E4
:1051F00002D20246084611464A0023D0C30D4A0097
:10520000DDB2120EAD1A202D35DA49020126490A07
:10521000F6058A19002C00D0524220214F1B11465E
:10522000B9402A411018C20D9A4221D0002C17D043
:10523000012D08DCDA05801AD20F8019D207DBB203
:1052400000F098FBF8BDDA05801A012340001B0628
:10525000C01880185A428018CA0F1043490007E04E
:105260004908C2071143DA05801A801940088018DE
:1052700000F078FBF8BD61000122511A001BF7E72E
:105280000122D2075140AAE70122D2075040A6E7E7
:10529000024670B54A40D30FDB0740002DD04A00CC
:1052A0002AD0010E140E000212020919400A520AF5
:1052B0008418E50104465443000A120A2E045043A0
:1052C000A4194219200CC543AA18120C0125AD03DC
:1052D000521C521912047F39240400D0521C10436E
:1052E00001D44000491EC2B20C06C0092018401C5F
:1052F0004008802A02D003E0002070BD4008400032
:10530000002900DA0020184370BD70B502464A40FB
:10531000D50F40004A00ED0740085208002814D07D
:10532000002A12D0C40DD30D41020120C005520243
:10533000490A520AE41A091812187D34914201D31D
:10534000641C00E04900002C01DA002070BD00233D
:10535000914201D3891A0343400849000028F7D13C
:1053600000290AD0914202D10121C90705E09142EA
:1053700001D2012101E00121C943E005C018401913
:1053800000F0F0FA70BD420005D04200120E524209
:105390008A4201DB00207047C905081870470000E9
:1053A000F0B507460846584087B0C00F0490480043
:1053B0000E46590040084908BC1A884105D23846B3
:1053C00031461E4617460B46024658004008104319
:1053D0004CD0300D039040055900400D490D05900B
:1053E000401A0290402872DA18030121000B0905C7
:1053F0000843019004980092002805D00199524278
:105400000020884100920190029840210A1A0199D7
:10541000009800F073FA05460C466B4607CB00F087
:105420008EFAC0197141039A0E0D0023D71756400A
:105430001A467A40164344D0049A002A2DD0029A84
:10544000012A039A15DC1205C01A9141012636057E
:10545000001C7141D20F059ED20700930192029663
:105460002A46234600F0CCFA07B0F0BD3846314654
:10547000FAE71605224A0F46B218C01AB7410121B1
:105480000905001C4F4100187F4111461818794149
:10549000E20F10436D19644113E0E2076D081543F4
:1054A0006408C2071443039A01261205C01A9141E9
:1054B0003605001C7141CE07400830434908C0182A
:1054C00051412A46234600F08EFACDE7FFE70498C3
:1054D00001224000C117121A00238B410498314663
:1054E000C417381AA141EEE730B40124E407634041
:1054F00030BC55E730B40124E407614030BC4FE7CD
:105500000000E0FFF0B51FB488B00B9909980024A3
:1055100048400999C00F490049080991C0070B99F3
:105520000090490049080B9109990898A64608433C
:105530001CD00B990A98084318D009980124400000
:10554000420D4800410D099824050003000B20433B
:1055500009900B980003000B20430B9050181C4936
:105560004018002201901446104605E00020014634
:105570000DB0F0BD032801DA034600E003239C468A
:10558000C11A0AAE0AE05F0008ADED5B4F00F75BA1
:105590007D430027AA187C41491C5B1E6145F2DD52
:1055A000410004AB5A522104120C0A43240C401C43
:1055B0000828DFDB01980290009970460191009065
:1055C000059B049A0799069800F01AFAD0E70000A4
:1055D0000DFCFFFFF0B50C465C4085B0E40FE4071E
:1055E00003944C000026640859009446490802467A
:1055F0000296224321D062460A431ED06200570D14
:105600004A000E032303550D012402462C492405AC
:10561000781B1B0B360B4018234326436146009032
:105620001C46501AB44103D30098401C009002E07D
:10563000921800985B41002803DA0020014605B06B
:10564000F0BD0020012109050746864611E06446A9
:105650001D46141BB54106D36546521BB341744623
:1056600007430C43A646CD07400849082843921833
:105670005B4105460D43EAD11046184313D06046FE
:10568000194650407140084306D06046101AB34195
:1056900006D20122002306E000220123DB0702E0FC
:1056A0000122D2435310009874460105381C614111
:1056B000029C039D0019694100F095F9BFE70000C5
:1056C000FD03000070B54B005B0803430BD04B009B
:1056D0005C0D002633466542B341D417AD1AA34191
:1056E00002DB0020014670BD12053018514170BD2B
:1056F000C217C10F504010B54018CA0796230021A9
:1057000000F038F910BD10B500229623114600F0C4
:1057100031F910BD0EB5C217C10F5040CA0740186D
:105720000021054B0293019200910A460B4600F0BE
:1057300067F903B000BD0000330400000EB5054951
:105740000291002100910A460B46019100F058F9A0
:1057500003B000BD33040000C20F4100400201232A
:10576000400ADB05D207090EC0187F2901DA0020A4
:105770007047962903DC9623591AC84001E09639F0
:105780008840002AF4D04042704741004002012284
:10579000400AD205090E80187F2901DA00207047DF
:1057A000962903DC9622511AC840704796398840E2
:1057B0007047000070B5CD0F4A0009030123090BA3
:1057C0001B0519430B4BED070024520D9A4201DAD9
:1057D000002070BD074B34339A4203DC9A1A00F064
:1057E0009DF802E00449511888402C43F1D0404212
:1057F00070BD0000FF030000CDFBFFFF4A0009035E
:105800000123090B1B051943094B10B5520D9A4290
:1058100001DA002010BD064B34339A4203DC9A1A99
:1058200000F07CF810BD03495118884010BD0000FD
:10583000FF030000CDFBFFFFC20FD207400040086E
:105840000BD0C10D0723DB01C91840020905400A2E
:105850001143C208400711437047002001467047BA
:1058600010B5002904DB0124E40740428C412146A5
:10587000002B04DB1C460123DB075242A3418B4271
:1058800000D1824210BD000010B5002904DB0124C4
:10589000E40740428C412146002B04DB1C460123D7
:1058A000DB075242A341994200D1904210BD000053
:1058B000CB0FDB07490010B5490802460A4307D061
:1058C0000A0D07240903E401090B121B002A01DC5D
:1058D000002010BDC900440F0C43C100E018D205E0
:1058E000801800F03FF810BD0122D207002800DB2D
:1058F000101A002900DB511A8142704710B5202A86
:1059000004DB0146203A9140002010BD9140202345
:105910009C1A0346E3401943904010BD10B5202A5D
:1059200004DB0846203AD040002110BD0B46D3408E
:10593000D0402024A21A91400843194610BD10B54A
:10594000202A06DBCB170846203A1041C1170B432B
:1059500006E00B461341D0402024A21A9140084390
:10596000194610BD002904DA401C490001D1400845
:105970004000704770B40024050C05D110240004C9
:1059800002D1002921D01124050E01D100020834D2
:10599000050F01D10001241D850F01D18000A41C39
:1059A000002801DB4000641C002908D020252E1BA4
:1059B0000D46F540A14000D00121294308430106CE
:1059C0001B1B000ADB1D02D5002070BC7047DB05E5
:1059D000181880180029F8DA401C4900F5D170BC6D
:1059E00040084000704710B5002B08DA0024401C26
:1059F000614192185B411A4301D14008400010BD3B
:105A0000F0B51FB482B005460C0003D0084604F080
:105A10007DFE02E004F07AFE20300246009021462E
:105A20002846FFF76BFF049B059A04460F46184370
:105A30001143084314D0184610431BD0009840214E
:105A40000A1A18460599FFF769FF05460E46009A9F
:105A500005990498FFF752FF084305D0012004E0A0
:105A60002046394607B0F0BD0020C11705430E435C
:105A70002C43374300990E986305401A7905E40AD0
:105A800000220C43FD0A0A3002D500200146E9E756
:105A90000105101969410C9C0D9D00196941FFF722
:105AA000A2FFDFE7FEB500231A461B1A8A4103DB7B
:105AB0000020014603B0F0BD4A000D0301212D0B6B
:105AC0000905520D0D43D10702D100186D41521E38
:105AD0005110FF31FF310131002704463E46384660
:105AE000009701910246012100200905FFF716FFEA
:105AF000C3197141F818324684468E464A416146C0
:105B00002846611A904104D36046241A954176468E
:105B10001F46241900986D41401C00903428E1DD97
:105B2000F91930467041091BA84103D20022D24323
:105B3000134601E00022134601980105381C71410B
:105B4000FFF751FFB6E70000064C0125064E05E0C1
:105B5000E36807CC2B430C3C98471034B442F7D38E
:105B6000FFF7B2FA08C8000828C8000870B58C18FA
:105B70000578401C6B075B0F01D10378401C2A118C
:105B800006D10278401C03E006780E70401C491CC8
:105B90005B1EF9D12B0705D40023521E0DD40B70C8
:105BA000491CFAE70378401CCB1A921C03E01D78CD
:105BB0000D70491C5B1C521EF9D5A142D8D30020A0
:105BC00070BD000038B50446064805490068FFF777
:105BD0008FFA604300E0401E00900028FBD138BDE2
:105BE00040420F0078010020F8B504460068816843
:105BF0008907890F012902D10168C90722D181686B
:105C0000114A10261140012500290ED1816829432F
:105C100081600120FFF7D6FF01F00EF807460CE087
:105C200001F00AF8C01B0A2807D9606D304360658F
:105C3000A06D2843A0650120F8BD20680068C0431E
:105C4000C007EDD10020F8BD170000801FB50B483C
:105C500000900B4801900B4802900B480390694656
:105C60000A4805F049F90A4A08481146083905F07A
:105C700031F800F055FA002004B010BD11C600083C
:105C8000EDC500084DC600084BC600088401002081
:105C90001000002010B500231A4603E0845CE318CE
:105CA0009BB2521C8A42F9D3D84380B210BD000087
:105CB00010B5034800F07CFD024800F079FD10BDEE
:105CC0005C1700201417002030B5446C1C252C40B4
:105CD0000125A540046C6560046863608368102B2F
:105CE000036803D099600068C26030BD9A600068A4
:105CF000C16030BD1449012048720A4602205E325C
:105D0000507203203C3A507204200E3A50720F48F1
:105D10000D4B0078087022310870203108770C494B
:105D20005A1C087858714978997123331871597140
:105D3000203318775977107551751A461E32107531
:105D40005175107651767047DC1100202701002034
:105D50004801002010B503F013FE202003F0BCFE24
:105D6000012005F033FB002003F0B6FE044805F0E7
:105D7000D1F9044805F080FC002005F0B5FC10BD09
:105D8000E800002083800000F8B50520012100070D
:105D900000F03EFF0025174C002800D06560164E2D
:105DA0000221304600F034FF00281BD10120207072
:105DB0001248808F00280ED00127BF0200223946EA
:105DC000304600F032FF0A2004F0F4FE012239468A
:105DD000304600F02AFF0A48656000880A214843DF
:105DE00008490880012000F04BFE022000F048FE28
:105DF000F8BD00006401002000040050DC0D00200C
:105E000034010020460100207047000010B5084909
:105E100000224A6107494B684C1523434B604B688D
:105E2000082423434B60C009C001026010BD00007C
:105E3000A4170020002002407FB500250C4606462E
:105E4000039500F0EDFDE009029003A9019600958D
:105E5000684600F07DFD002804D000F0B5FD00206C
:105E600004B070BD00F0B0FD0120F9E710B50023CB
:105E700002E0C45CCC545B1C9342FAD310BD00001A
:105E800010B5214A00219069C305204804D5416915
:105E9000022319434161911593699B0505D5436917
:105EA0000124234343616302194393695B0505D5CC
:105EB0004369082423434361E301194393691B05A4
:105EC00005D543690424234343616302194393695D
:105ED0009B0405D54369102423434361630219439E
:105EE00093699B0304D5446920231C4344611943EF
:105EF0009369DB0305D54369402423434361A00232
:105F00000143916110BD000000200240A417002051
:105F100070B5054600F090FE0646184C0AE0681C75
:105F200008D0002D04D000F087FE801BA84201D9C4
:105F3000032070BDA069C007F1D1A069800701D519
:105F40000220A061A069C00511D4A06980050ED40B
:105F5000A06940050BD4A069000508D4A06980049D
:105F600005D4A069800302D4A069C00303D5FFF75C
:105F700087FF012070BD002070BD0000002002409E
:105F8000F8B51746002605460C4600F049FD09E025
:105F900029460220226800F025FD002804D1241D96
:105FA0002D1D361DBE42F3D300F00EFDBE4201D2C0
:105FB0000020F8BD0120F8BD10B5084902460020B8
:105FC000054B497905E044001C5B944203D0401C1A
:105FD000C0B28842F7D310BD6813002070000020C3
:105FE00010B500F01AFE10BD10B5094801F044F8D4
:105FF00080B2FFF7A3FB074A074BFFF783FA0022A3
:10600000064BFFF7E7FAFFF7F9FB80B210BD00007F
:10601000C8150020F853E3A59B843E4000408F4004
:1060200070B5394A394900208300401CC0B2CA50BB
:106030001428F9D3374936488A7F0275C97F4175DC
:1060400035490A780276497841763149052013317D
:1060500048720A2005F000FB7D20C00005F016FB09
:106060002B49002213310C2005F0E0FB00210C200D
:1060700005F0EEFB022005F03FFB284D254C0021EA
:106080000F2005F069FA28422063F8D0206B411CEC
:1060900038D0400435D58122D20100210F2005F0EF
:1060A0009AFB0021102005F057FA41061748490EC7
:1060B0000022C43805F086FA144DC43D687A0528DC
:1060C0001FD102221449681DFFF77CF8002818D15F
:1060D0001048AE7C66710422691C4C30FFF74EF804
:1060E00029461331084672000D465130FFF746F835
:1060F00060792946420005484838FFF73FF80320F9
:10610000207070BD04F076FBFFFF0100C813002073
:106110003D120020700000204801002000D02724FC
:1061200010B5144C1448224610321146083904F0B8
:10613000D1FD0022114BE168A068FFF74BFA104A2D
:10614000104B05F0F5FC00220F4BFFF7D3F90022AE
:106150000E4BFFF7D7F9FFF7ABFB20600022134689
:10616000E168A068FFF77CFB01D0206810BD00202B
:10617000206010BD000000208401002000AA8F4094
:106180006C45D9CC955BC83F0000F03F40A5E54089
:1061900010B5084800F096FA0A21064800F032FAD5
:1061A000044800F01DF9800503D5024800F01AF9F3
:1061B00080B210BD6C150020F8B52F4D00220121D2
:1061C000284600F032FDFFF7E3FFFFF79CFA2B4E65
:1061D0003146FFF79AF82A4C0122A0601146284662
:1061E00000F023FD2749A068002588423EDB207887
:1061F000254F002815D02570FFF7CAFFFFF783FA57
:106200003146FFF782F8A060FFF716FB00223B46FD
:10621000FFF76AF900221D4BFFF774F9FFF748FBFF
:106220006060A068FFF708FB00223B46FFF75CF9BF
:10623000174A184BFFF766F906460F466068FFF7E6
:10624000FBFA134A144B5242FFF75CF932463B46C5
:10625000FFF7A6F8FFF72CFB10496060884201DDCC
:10626000616004E0FF21C905C84200D36560606831
:10627000FFF78BFAC0B2F8BD0004005000401B4489
:10628000480000200000604000000C4000E0644036
:106290003333333333B33040CCCCEC3F0000C8420F
:1062A000F8B5054604464035287C0026012808D06C
:1062B00001202874206881688907890F01290ED17F
:1062C00001E00220F8BD0168C90708D0606D2021F7
:1062D000084360650126002028743046F8BD616DD2
:1062E000FF2201329143022211436165C16889078F
:1062F000890F0091C16889088900C16020688168A0
:1063000092071143816000F097FC07460EE000F011
:1063100093FCC01B0A2809D9606D02218843102113
:1063200008436065002028740120F8BD206880685B
:106330000028ECDB2068C168009A1143C160606DE1
:1063400080088000401C6065C5E70000F8B506467F
:106350000D464036317C01290DD001213174016890
:106360008A68520709D5416D2022114341650020FA
:1063700030740120F8BD0220F8BD174B6A68D805BB
:1063800047109A42154C8A6A2B6812D05B035B0B4C
:106390001A438A622968490305D5A1680143A160AF
:1063A0000A20FFF70FFC2868800312D5A068384345
:1063B0000EE05B035B0B9A438A622968490302D5AE
:1063C000A1688143A1602868800302D5A068B84312
:1063D000A06000203074F8BD0110000000270140CB
:1063E000406D70470068006C7047000070B5040095
:1063F00006D0606D264600254036002802D006E013
:10640000012070BDA5653574204600F0D3F8606D9D
:10641000C00603D421688868400705D5606D102147
:10642000084360653574EBE7606DFF2201329043ED
:1064300002221043606588688207920F5B48012A38
:1064400002D10A68D2072BD1032362689B079A42C4
:1064500005D05B429A4202D05B009A4209D10A6998
:10646000920092080A6121680A6963681A430A6106
:106470000CE00A69920092080A6181680F22920476
:106480009143816081686268114381602168CA68B4
:1064900018239A43CA602168CA68A3681A43CA606D
:1064A000816801225206914381608168A28E520662
:1064B0001143816020688168C90004D48168012289
:1064C0001207114381602068C168394A1140C160D8
:1064D0002069E168022825D00020014320462030B1
:1064E0000278037B52035B001A431143226B114372
:1064F000A26992031143E269D20311432268D3686F
:106500001943D160616A0A46FF3AC23A05D0A26ACD
:1065100011432268D3681943D16042780121012ACE
:1065200002D00BE00420D8E70078002823D0606D6B
:10653000202210436065A06D0843A065E06B012830
:1065400020681FD00169C90703D0016949084900C3
:10655000016120684169C908C90041612068416939
:10656000A26B11434161A565606D80088000401CED
:106570006065002070BD2068C26801231B041A43B7
:10658000C260DBE70269FF239B009A430261206837
:106590000269236CA66C1A43636C33431A4302618D
:1065A000206802690A430261D3E700000027014026
:1065B0001902FEFF10B586B0044614216846FEF7A6
:1065C000F6FD0E492068884216D10D48416B4215F0
:1065D00011434163C16A01221143C162C06A694625
:1065E00010400590022000900320019000200290AE
:1065F0000520000700F050FA06B010BD002401404D
:1066000000100240F8B504464069254640350E4664
:1066100008280BD02068C068C00709D0606D202111
:1066200008436065002028740120F8BD082700E0B9
:106630000C2700F001FB009011E0701C0FD0002E21
:1066400005D000F0F9FA0099401AB04207D9606D00
:10665000042108436065002028740320F8BD2068E9
:1066600000683842E9D0606D012149020843606545
:106670002068C16809058A0F0C21002A1BD120223D
:10668000125D002A17D10268120714D582685307D9
:106690000122002B08DB43688B434360606D1302CB
:1066A00098431043606506E0606D202318436065E1
:1066B000A06D1043A065A069002801D12068016089
:1066C0000020F8BD70B5044621680020896849079C
:1066D00021D425464035297C01291CD0012129746B
:1066E000E169012904D02046FFF77EFA002811D184
:1066F000616D0A4A1140FF22013211436165002198
:10670000A165297422681C21116021688A6804230C
:106710001A438A6070BD022070BD0000FEF1FFFFC9
:1067200030B5014620314A790023022A04D00422E0
:10673000C2630B71012030BD026814680E25AC43A2
:10674000146002681468640864001460446C1C22BD
:10675000144001221546006CA54045604A71184658
:106760000B7130BD70B50024014620314A79022AF0
:1067700003D00421C163012418E0026813680E25C8
:10678000AB431360026813685B085B001360436CE3
:106790001C221340012215469D40036C5D604A7126
:1067A00000220A71816B002900D08847204670BD05
:1067B000F0B4016C0D6801680C68466C1C2304225F
:1067C0001E401746B7402F420ED067070CD50C6805
:1067D000A40602D40C6894430C60416C19408A40B2
:1067E000016C4A60016B1AE00227B74002462F4055
:1067F0002032002F17D0A70715D50C68A40605D4A2
:106800000C680A25AC430C6001215171446C0221D3
:106810001C40036CA140596000211171C16A00291C
:1068200018D0F0BC08470827B7402F4212D02407E1
:1068300010D50C680E25AC430C60446C01211C4043
:106840000B46A340046C6360C16351710021117158
:10685000416BE4E7F0BC704770B504003CD01F48C2
:10686000256814212818FEF743FC800060641C484A
:1068700020640221204620300246417129681948CF
:10688000E3680140A06866691843236933431843ED
:10689000A3691843E3691843236A1843084328602F
:1068A0000121A0688903884210D00D488030836A96
:1068B000656C1C210D400F26AE40B3438362656CAE
:1068C00063680D40816AAB400B4383620020E06344
:1068D00001215171107170BD012070BDF8FFFDBF25
:1068E000000002400F80FFFFF8B504468C462030C0
:1068F00001790025012909D0012606714179002777
:10690000012905D0077102252846F8BD0220F8BDEF
:1069100002214171E763206801684908490001606C
:1069200061462046FFF7D0F9206B002820680168F7
:1069300001D00E2205E00422914301602068016825
:106940000A22114301602068016831430160DBE7DE
:10695000F8B51A4E0546307C0F46012807D00120B5
:1069600030741748FFF7D4FA010002D021E002206A
:10697000F8BD0020C04338606C6814E02046FFF783
:1069800045FA0F48FFF7C4FA01460E48426808234B
:106990009A434260426843159A434260002901D0FD
:1069A0003C6006E08034A8686A68C0018018A04294
:1069B000E4D8002030740846F8BD0000A417002079
:1069C00050C30000002002400548416802221143E4
:1069D000416041680122114341600020704700007E
:1069E00000200240F8B50C4C1646207C0F460128CA
:1069F00008D0012020740948FFF78AFA00250028F2
:106A000002D006E00220F8BD65613E600348FFF752
:106A10007FFA2574F8BD0000A417002050C30000C1
:106A200011484168C9070BD0EFF3108172B60F4AC5
:106A3000C2600F4AC26081F310884168C9070ED155
:106A4000416889070DD5EFF3108172B6094A0261DA
:106A5000094A026181F310884068800701D501204E
:106A6000704700207047000000200240EFCDAB8946
:106A700005040302BFAE9D8C161514137047000069
:106A800010B504494A69024202D04861FFF7F6FF97
:106A900010BD000000040140FCB500230124A2E069
:106AA00027462A469F403A406FD04D68012D05D0B9
:106AB000022D03D0112D01D0122D16D18568032689
:106AC000AC465D00AE46AE406546B543AC46CE68CA
:106AD0007546AE4065462E43866046680D79BE43D6
:106AE000ED06ED0F9D4035434560C6685F00032508
:106AF000BD40AE46AE4335468E68BE402E43C660AE
:106B00004E68022E01D0122E14D1DE08B6003618BF
:106B10000196366A5D07B446EE0E0F25B540009625
:106B20006646AE43B4460D69009EB54066462E43A8
:106B3000019D2E6206687546AE430D79AD07AD0F17
:106B4000BD40354305604D68ED004BD5294D6E6B5A
:106B500026436E639E08284DB6007519AC46AD6895
:106B60009E07360F0F27B740BD4305273F07B842A2
:106B700001D1002715E0214FB84201D1012710E0D3
:106B80001F4FB84202D102270BE02BE01D4FB84245
:106B900001D1032705E01C4FB84201D1052700E0D1
:106BA0000627B7402F436546AF60184D2E684F68E3
:106BB0009643FF0300D516432E606E684F689643D8
:106BC000BF0300D516436E60AE684F689643FF0260
:106BD00000D51643AE60EE684F689643BF0200D5FD
:106BE0001643EE605B1C0A681546DA4000D057E792
:106BF000FCBD0000001002400000014000040050F5
:106C000000080050000C0050001C0050000401401F
:106C10000069084000D001207047426913460B40CC
:106C20001B0491430B4383617047002A01D08161AB
:106C3000704781627047000001488068704700001B
:106C40006C010020024881680278891881607047D1
:106C50006C01002010B5084800240168402211434F
:106C60000160204600F00AF8002801D0012401E06C
:106C700000F04CFA204610BD0020024070B50446DA
:106C80000D4D7D202978C000FEF732FA01460B48F1
:106C90000068FEF72DFA00F035FF002809D1042C1A
:106CA00007D200222146401E00F058FA00206C60F6
:106CB00070BD012070BD00006C0100207801002033
:106CC00070477047F8B5654CA078401CA070012053
:106CD0002071A08B401CA0836148008802F0B8FEA0
:106CE000208AFEF710FD01467F20C005FEF70DFB50
:106CF0005C4D06462968FEF772FA28600120A16AF9
:106D0000C005814201DA084603E03046FEF7BCFACE
:106D1000A062FF21C9050025C84200D3A5626078A2
:106D200000280BD102215048FFF772FF02004F49A3
:106D30004F4817D00022FFF778FFA56302214A4889
:106D4000FFF766FF4B4E002855D0A563B08AFEF7CB
:106D5000DAFC444F3968FEF7C7FD5FD2464901208F
:106D600008705DE00122D1034148FFF75EFF208AF1
:106D7000FEF7C9FC01467F20C005FEF7C6FAA16BED
:106D8000FEF72DFA3D49A0638842D7DD3948012737
:106D9000F926403000900A213046FEF7A9F9002973
:106DA00003D132493248FFF71BF902212E48FFF781
:106DB0002FFF002801D0002701E0002F12D102216F
:106DC0002948FFF725FF00280CD104F079FE00992F
:106DD0000120888005F0D0FB642003F0EBFE2949F8
:106DE0002748C8600A2003F0E5FE3046761EF6B25A
:106DF0000028D0D1A2E7208AFEF785FC01467F203B
:106E0000C005FEF782FAA16BFEF7E9F91E49A063FF
:106E100088429BDB1B491A48C86097E716480570F3
:106E2000708F401EFEF764FC3968FEF75DFD06D8E2
:106E30006079002803D015490120087001E013484B
:106E40000570708FFEF75FFC3968FEF74DFD04D2C8
:106E50006079002801D004F0F7FDF8BD240100207E
:106E60008C00002068010020000400500080000019
:106E700000000050DC0D00207600002000004040A3
:106E80000400FA0500ED00E00000A04084000020AE
:106E9000704770B5040010D0022025462035A87335
:106EA000204601F0F9FCA87B032805D0204600F01D
:106EB000B9F80020A873687370BD012070BD7047D9
:106EC000704710B5044600680168C943C90708D176
:106ED0008168C943C90704D1012141602046FFF7F9
:106EE000F1FE20680168C943890708D48168C94355
:106EF000890704D4022141602046FFF7E1FE2068A3
:106F00000168C943490708D48168C943490704D4C3
:106F100004214160204600F0F7F820680168C94369
:106F2000090708D48168C943090704D408214160CE
:106F30002046FFF7ADFF20680168C943C90608D4A1
:106F40008168C943C90604D4102141602046FFF777
:106F5000B8FE20680168C943890608D48168C9431E
:106F6000890604D4202141602046FFF7A9FF20684C
:106F70000168C943490608D48168C943490604D455
:106F8000402141602046FFF79AFF10BDF8B504008C
:106F900005D025462035A87B002802D006E0012038
:106FA000F8BD00206873204600F04EF80220A87358
:106FB0002068C26884466368012B01D106208243A1
:106FC00016486169814202D0072040038243002BAA
:106FD00001D1D82082431248A668024018463043A7
:106FE000676A266A3E433043A66A30431043002B4B
:106FF00002D0012B04D005E02369E2691A4300E0C6
:10700000E2681043054A914202D0A2691143084345
:107010006146C8600120A8730020F8BDFFFF000092
:10702000F8F119FF10B500680549884207D10548F5
:10703000816B4900490881630D2000F073F810BD91
:10704000007C00400010024010B5006808498842EA
:107050000CD10848816BC2041143816300220121D5
:107060000D2000F07BF80D2000F06CF810BD000042
:10707000007C0040001002400068C06970470000BA
:10708000F8B504460220254620351746A8731D484A
:107090000268C3041A4302602068C2689B121A4344
:1070A000C260206802690126324302612268102012
:1070B0005060206881611021204601F05DFC0328AA
:1070C0001FD02168082048602068476108212046B9
:1070D00001F052FC032814D0204601F0DDFBA87B10
:1070E00003280ED0206881683143816020680169DF
:1070F0003143016120680169042211430161AE73CB
:107100000020F8BD00040140704700000448416BB6
:10711000012211434163816B020411438163704773
:1071200000100240002809DBC106C90E012088407A
:1071300003490860BFF34F8FBFF36F8F70470000A4
:1071400080E100E0002805DBC106C90E012088406F
:10715000014908607047000000E100E010B503F04D
:1071600027FB10BD02494A6882434A60704700000D
:1071700000700040024801688215114301607047A9
:107180000070004002494A6802434A6070470000AC
:107190000070004005480168022211430160044864
:1071A000016904221143016130BF70470070004043
:1071B00000ED00E0F0B5154A1368154D54152D6A21
:1071C0002340ED07ED0F002B04D0002D02D01668F0
:1071D000A64316601668B608B600064316600D484A
:1071E000076904263743076101290DD040BF20BF3E
:1071F00020BF0169B1430161002B04D0002D02D0F2
:10720000106820431060F0BD30BFF2E7007000400E
:107210000000014000ED00E0F8B5044600780027CA
:10722000534D800671D5524E403EB06BC00004D421
:10723000B06BA9050843B06301274E480168C90532
:1072400011D40168821511430160FFF7F5FC00902D
:1072500005E0FFF7F1FC0099401A642837D845484B
:107260000068C005F5D532680321090560680A4049
:107270000140914208D08103890F032904D131686C
:10728000890301D50120F8BD2A69032109040A40B8
:1072900022D0084090421FD0207880061CD5286953
:1072A0002A6988430121C9040A432A612A698A4359
:1072B0002A612861C0050FD5FFF7BEFC009008E0E9
:1072C000FFF7BAFC0099411A2B48814201D90320EB
:1072D000F8BD28698005F3D561688803800F03280D
:1072E00005D132680005824301400A4332602869B3
:1072F000032261681204114008432861002F04D062
:10730000B16B012000078143B1632078C00705D02D
:10731000E868A168800880000843E860207880075A
:1073200005D5E8680C218843E1680843E8602078C7
:10733000400706D5E868032189028843216908438C
:10734000E8602078000706D5E86803210903884330
:1073500061690843E8602078000606D5E8680321E3
:1073600089048843A1690843E8600020F8BD000053
:10737000401002400070004088130000F8B50E462F
:10738000050038D05E480068C007C00FB04214D274
:107390005B4C20684008400030432060FFF74CFC05
:1073A000074605E0FFF748FCC11B564881427AD8E2
:1073B0002068C007C00FB042F4D12878524C800733
:1073C00005D5E068F0218843A9680843E060287883
:1073D000C00752D06868022806D0032807D0216869
:1073E00001280AD0890504E02168890301E02168A9
:1073F0008901002903DB0120F8BD4907F9E7E168AD
:10740000890889000143E160FFF716FC07466868B8
:1074100002280AD0032814D001281ED029E0FFF743
:107420000BFCC11B374881423DD8E0680007800F44
:107430000228F4D121E0FFF7FFFBC11B3148814254
:1074400031D8E0680007800F0328F4D115E0FFF77A
:10745000F3FBC11B2B48814225D8E0680007800F51
:107460000128F4D109E0FFF7E7FBC11B2548814261
:1074700019D8E0680007800FF5D121480168C907D5
:10748000C90FB14217D90168490849003143016069
:10749000FFF7D2FB074608E005E0FFF7CDFBC11B75
:1074A0001848814201D90320F8BD15480068C0077B
:1074B000C00FB042F1D12878400706D5E068072117
:1074C00009028843E9680843E0602878000707D587
:1074D000E0680721C90288432969C9000843E060C0
:1074E00000F03AF8E168094A0906090F515CC84002
:1074F0000749086007480068FFF7C0FBF8BD0000B7
:1075000000200240881300000010024052C700080B
:107510007801002070010020044805490068C9680E
:10752000044A4905490F515CC84070477801002062
:10753000001002406BC70008044805490068C9688C
:10754000044A8904490F515CC84070477801002003
:10755000001002406BC7000870B51A4AD3681A4978
:107560000C2018408D0004280CD04E00082810D0A4
:107570000C2810D050680004410F0120C003491CA2
:10758000884070BD1068C00601D5084670BD284609
:1075900070BD304670BD98020C4C000F205C1B0281
:1075A0009C0FD368641CDB0301D5314603E01268ED
:1075B000D20600D4294603F0C0F822460023FDF786
:1075C000ADFD70BD0010024000093D0062C700081B
:1075D000FEB505007ED0FE4CE7680C20E66807404B
:1075E0000120000406402878C00747D0082F05D0A6
:1075F0000C2F0AD101200004864206D120688003A6
:107600003CD568680028E5D038E0012069680004AE
:10761000814203D121680143216011E00523012249
:107620001B0492049942216802D111432160F1E7C1
:1076300081432160216801400091206890432060CF
:10764000686800280DD0FFF7F7FA009005E0FFF713
:10765000F3FA0099401A64287BD820688003F6D595
:107660000CE0FFF7E9FA009005E0FFF7E5FA009972
:10767000401A6428F0D820688003F6D42878800760
:1076800056D50923E868042F0DD00C2F01D1002E08
:1076900009D000283CD02168994301432160FFF7BD
:1076A000CBFA064628E02168490701D5002891D089
:1076B00061681F22120291432A691202114361601C
:1076C0002168994301432160FFF746FFE1680906FD
:1076D0000A0F00E08BE1BF49895CC840BE490860E1
:1076E000BE480068FFF7CAFA002873D120E0FFF710
:1076F000A3FA801B0228AFD820684007F7D560683E
:107700001F210902884329690902084360600FE0CC
:107710002068400840002060FFF78EFA064604E02B
:10772000FFF78AFA801B022896D820684007F7D412
:107730002878C00660D5002F0CD0A86900284AD050
:107740002068FF21013108432060FFF775FA0646E3
:107750002EE0C1E02068800502D5A8690028A6D0E7
:107760006068072149038843296A084360606068AC
:10777000297F0002000A090608436060286A410B5D
:107780000120C003491C8840E16809060A0F91499D
:10779000895CC8409049086090480068FFF76EFA1D
:1077A000002817D128E0FFF747FA801B0228A2D84B
:1077B00020688005F7D56068072149038843296A56
:1077C000084360606068297F0002000A09060843D8
:1077D000606011E0E2E02168FF2001308143216018
:1077E000FFF72AFA064604E0FFF726FA801B022874
:1077F00072D820688005F7D42878794E000724D500
:1078000068690028306910D0012108433061FFF712
:1078100013FA009005E0FFF70FFA0099401A0228CA
:107820005AD830698007F6D50FE040084000306133
:10783000FFF702FA009005E0FFF7FEF90099401A01
:10784000022849D830698007F6D42878400766D5E1
:1078500000200290A06BC00006D4A06B0121090794
:107860000843A063012002905E480168C90511D455
:107870000168821511430160FFF7DEF9009005E011
:10788000FFF7DAF90099401A642825D855480068AE
:10789000C005F5D5FF20AA680130824203D13169C5
:1078A0000143316111E001218902002A07D005233B
:1078B0001B029A4203D132690A433261EFE732690F
:1078C00082433261306988433061A868002810D053
:1078D000FFF7B2F9009008E05FE0FFF7ADF901466D
:1078E0000098091A4048814257D830698005F4D57C
:1078F0000DE0FFF7A1F9009006E0FFF79DF9009970
:10790000411A3948814248D830698005F5D4029837
:10791000002804D0A06B012109078843A063686A8E
:10792000002866D00C2F3ED001263606022820689B
:1079300005D0B0432060FFF77FF905462FE0B04344
:107940002060FFF779F9074604E0FFF775F9C01BDF
:10795000022822D820688001F7D4E96AA86AE26880
:107960000843296BFD231B049A4311430843E0603D
:10797000206830432060FFF75FF9054604E0FFF719
:107980005BF9401B022808D820688001F7D530E059
:10799000FFF752F9401B022801D90320FEBD2068E1
:1079A0008001F5D425E00128F8D0E0680121090420
:1079B000AA6A014091421AD10F218904EA6A014062
:1079C000914214D1032189050840296B88420DE0BA
:1079D0000010024052C7000878010020700100200A
:1079E00040100240007000408813000001D00120C8
:1079F000FEBD0020FEBDF8B504000ED0FF27606A72
:107A00000537002500280AD02561656126464036E5
:107A1000A562707C002807D00AE00120F8BD6068EC
:107A2000B842F3D0E561F1E73574204600F03EF846
:107A3000022171742068026840239A430260212366
:107A4000A26860689B021A4038401043E3688A02CB
:107A50001340184323690B40217D1843C907C90F00
:107A60000843A169931019400843E169382319407C
:107A70000843216A802319400843A16A93001940F2
:107A8000084321680860A0690421000C0840616A6D
:107A9000102319400843216848602068C169914358
:107AA000C1616565012070740020F8BD10B586B015
:107AB000044614216846FDF77AFB10492068884285
:107AC00019D10F48416B821411434163C16A0122ED
:107AD0001143C162C06A002110400590E02000906F
:107AE0000220019003200390029104910520694631
:107AF0000007FEF7D1FF06B010BD000000300140C6
:107B000000100240094910B5401E884201D90120E9
:107B100010BD074C60610321081F02F049FE0020E0
:107B2000A06107202061002010BD0000FFFFFF00C2
:107B300000E000E0F0B502462032137E012B1ED09B
:107B4000012515760223537606687468B36870279A
:107B5000BC430F68274377600068AC07A04205D09C
:107B6000084CA04202D0084CA04204D180244968AD
:107B7000A34319438160557600201076F0BD0220A2
:107B8000F0BD0000000801400014014070B5050080
:107B900005D02C462034607E002802D006E001206B
:107BA00070BD00202076284600F010F80220607694
:107BB000291D286802F014F80120A077A076E0764D
:107BC000207760776076002070BD0000006801219A
:107BD0008907884204D10348816B012211438163E4
:107BE0007047000000100240F8B5054604462035F5
:107BF000287E012817D001262E760220687622687A
:107C000090687727FF23B8431B02984390600A6867
:107C1000502A31D00EDC202A4BD006DC002A48D076
:107C2000102A3AD145E00220F8BD302A41D0402A3E
:107C300033D136E0602A27D0702A12D00120000309
:107C4000121A2AD0824228D1CB684A6889682068F3
:107C500001F0FFFF206881680122920311438160D7
:107C60001BE0CB684A688968206801F0F2FF216850
:107C700088683843886010E0CA684968206802F064
:107C800062F85021206806E0CA684968206802F05E
:107C90006BF86021206801F0E7FF6E7600202876FF
:107CA000F8BDCA684968206802F04DF84021206894
:107CB000F1E711462068EEE710B586B004461421BE
:107CC0006846FDF774FA012120688907884212D1BD
:107CD0000A49CA6A02200243CA62C96A0190014085
:107CE000059141020091002102910391049069469F
:107CF0000348FEF7D1FE06B010BD000000100240A0
:107D000000040050F8B5064604462036307E0D4685
:107D100001280BD0012008273076002A08D0042A39
:107D200016D0082A2AD00C2A4DD137E00220F8BDFF
:107D3000206801F0A1FF20688169394381612068D2
:107D4000816904229143816120688169EA6812E0B7
:107D5000206801F0A9FF206881690122D202114345
:107D6000816120688269012189028A4382612068D9
:107D70008169EA6812021143816124E0206801F000
:107D8000ACFF2068C1693943C1612068C169042220
:107D90009143C1612068C169EA6812E0206801F07E
:107DA000B7FF2068C1690122D2021143C161206876
:107DB000C269012189028A43C2612068C169EA68F7
:107DC00012021143C16100203076F8BD70B5050084
:107DD00005D02C462034607E002802D006E0012029
:107DE00070BD00202076284600F00FF80220607653
:107DF000291D286801F0F4FE0120A077A076E07626
:107E0000207760776076002070BD704770B50546BA
:107E10002C4602202034002908D004290BD0082940
:107E20000ED0627F012A10D0012070BDA27E012AEF
:107E3000FAD1A0760AE0E27E012AF5D1E07605E0EB
:107E4000227F012AF0D1207700E0607701222868A4
:107E500001F0F2FE0122286892070121904205D02C
:107E6000074A904202D0074A904204D182685207E2
:107E7000520F062A02D002680A430260002070BD39
:107E8000000801400014014070B504460D4600682A
:107E9000002201F0D1FE2068016A0C4A114203D190
:107EA000016849084900016001202034002D06D0F6
:107EB000042D06D0082D06D06077002070BDA07676
:107EC000FBE7E076F9E72077F7E700001111000003
:107ED0007047704770470000F8B502680446D069E3
:107EE00011689668814B05461D402023002D6CD0FB
:107EF000F7077F4DFF0FBC460D402F4379D0254635
:107F0000C7078035002F06D0CF0504D5012717629B
:107F10002A683A432A60820708D5F20706D0276804
:107F200002223A622A6804273A432A60420708D5A7
:107F3000F20706D02668042232622A6802263243FB
:107F40002A6002070AD50A461A406646324305D01F
:107F50002668082232622E6816432E60020508D574
:107F60004A0106D501222668D20232622A681A43E3
:107F70002A602A68002A30D0800606D5880604D5F3
:107F8000616E002901D020468847286821688968E9
:107F9000490602D42821084225D0204602F013F9D0
:107FA00020688168490619D5826840218A43826029
:107FB000206F002812D04F498163206FFEF7D2FB5B
:107FC00000280AD0206F816B06E0850611D58D064A
:107FD0000FD5616E77E020468847F8BD2046FFF751
:107FE00079FFF8BD05E02046FFF774FF0020286008
:107FF000F7E7256E012D56D1C50654D5CD0652D5CD
:1080000010261662206881682546490640350029F9
:108010002ADA226F116849680904090CE1D02F8B14
:108020008F42DED9698311680968890617D401680F
:1080300032019143016020688168490849008160EC
:1080400020688168402291438160E36700202066B8
:1080500020680168B1430160206FFEF761FB288B47
:10806000698B401A81B21AE0298B6A8B891A6A8B54
:1080700089B2002AB5D00029B3D00268FF25213586
:10808000AA43026020688268520852008260E36757
:1080900000202066606620680268B24302602046C5
:1080A000FFF716FF9DE7C50208D5750206D501202A
:1080B000000510622046FFF70CFF92E7050605D584
:1080C0000D0603D5A16E002985D18AE7400688D523
:1080D000480686D5116820464024A1431160836775
:1080E0000021816600F043F97BE700000F080000E3
:1080F00020010004EDA0000810B5040003D0A06F1B
:10810000002802D007E0012010BD00217420015595
:10811000204600F027F82420A0672068016849085D
:1081200049000160204602F0A1F80128ECD0606A05
:10813000002802D0204601F0B9FE206841680922DB
:10814000D20291434160206881682A229143816074
:1081500020680168012211430160204601F00CFFF4
:1081600010BD0000F0B587B0064614216846FDF743
:108170001EF82C493068884251D12B48416B0122AE
:10818000920311434163C16A01221143C162C06A73
:108190000025104005900320400200900220032794
:1081A00001A9A1C104200490052069460007FEF73B
:1081B00073FC1F4C1D48A560E56081C48027E56005
:1081C000A7602020256160610002A0611848083C7A
:1081D000FEF742FB002801D0FDF716FE3467A662C9
:1081E000144C12482146143820600320606010208F
:1081F0000831A1C16561A561E56120462562FEF7F0
:108200002BFB002801D0FDF7FFFDF46600220121C1
:108210001B20A662FEF7A2FF1B20FEF793FF07B00C
:10822000F0BD000000380140001002403000024064
:10823000141700205C17002070B5C36F202B27D1C6
:1082400000290BD0002A09D0012483682403A3420B
:1082500006D10369002B03D1CB0701D0012070BDEB
:10826000034660331C7D012C12D001241C750023B1
:108270000366084C0368A34207D05C68240204D557
:108280001C680125AD062C431C6002F0EFF870BDA0
:10829000022070BD0048004070477047FFB504469B
:1082A000806F83B017460D4620285ED1002D0AD07E
:1082B000002F08D0A168C001814207D120690028A1
:1082C00004D1E80702D0012007B0F0BD204660309D
:1082D0000090007D012848D0009801210175002000
:1082E000802108512120A067FEF7A6FC26464036D3
:1082F0000190378277820120A1680003814202D178
:108300002069002805D02F46002500990020087517
:1083100011E00027F9E700228021204602F0ECF866
:10832000002815D1002F15D02168387888627F1C6D
:10833000708A401E7082708A019B00280698009007
:10834000E9D100224021204602F0D6F8002808D0CA
:108350000320B9E728882168C005C00D8862AD1CDC
:10836000E6E72020A0670020AEE70220ACE77047D8
:10837000034D044C04A002F0BFF9E560FAE70000E9
:108380000400FA0500ED00E0486172644661756C16
:10839000745F48616E646C65722E0D0A0000000007
:1083A00070B586B014216846FCF701FF104801241F
:1083B000418B002900D14483408B012807D002283B
:1083C00003D100F003FCFDF741FC06B070BD0122B3
:1083D000084E950229463046FEF727FC00210291FF
:1083E00003910095019469463046FEF755FBECE792
:1083F000240100200004005010B5052424070022A9
:1084000004212046FEF711FC002208212046FEF739
:108410000CFC0A2002F0D5FB012204212046FEF7C5
:1084200004FC0A2002F0CDFB002204212046FEF7C6
:10843000FCFB10BD10B505242407002204212046B2
:10844000FEF7F3FB012208212046FEF7EEFB0A208F
:1084500002F0B7FB012204212046FEF7E6FB0A20CA
:1084600002F0AFFB002204212046FEF7DEFB10BD28
:10847000F8B50024052607462546360700220421C4
:108480003046FEF7D2FB0A2002F09BFB01220421BA
:108490003046FEF7CAFB6006040E08213046FEF7A0
:1084A000B7FB002801D0641CE4B2052002F089FB70
:1084B0006D1CEDB2082DE1D3002F03D0FFF79CFF18
:1084C0002046F8BDFFF7B6FFFAE770B5052605466A
:1084D0003607002204213046FEF7A7FB0024E809F6
:1084E00001D0012200E0002208213046FEF79DFB6A
:1084F0006806050E0A2002F064FB012204213046C2
:10850000FEF793FB0A2002F05CFB002204213046B8
:10851000FEF78BFB0A2002F054FB641CE4B2082C2B
:10852000DDD370BD10B505242407012208212046A3
:10853000FEF77BFB012204212046FEF776FB00229A
:1085400008212046FEF771FB0A2002F03AFB0022C8
:1085500004212046FEF769FB10BD10B50524240751
:10856000002204212046FEF760FB0022082120465D
:10857000FEF75BFB0A2002F024FB012204212046C7
:10858000FEF753FB012208212046FEF74EFB0A208E
:1085900002F017FB10BD70B505252D070024012240
:1085A00008212846FEF741FB062002F00AFB0122C3
:1085B00004212846FEF739FB062002F002FB07E003
:1085C000641CE4B2FA2C03D9FFF7C7FF012070BD89
:1085D00008212846FEF71CFB0028F1D100220421C7
:1085E0002846FEF722FB002070BD0000F8B501F020
:1085F000F5FC01F02FFD5B480068C069FDF7F4FC55
:10860000594C5A49A082898F594E0025002931D0F2
:10861000A26A730357499A4202DB02220A7000E001
:108620000D700A7801218902002A05D0012A0ED096
:10863000022A10D0032A1DD1608B01282ED00228D7
:1086400018D1484808214038FFF71EFC12E0FF22ED
:10865000F5329042F0D2608B01281DD0022804D060
:1086600008E03046FEF7E1FA04E03E4808214038D1
:10867000FFF7CCFBFDF7A0FD20700121C9023046B9
:10868000FEF7C6FA0127FF0300282DD03A480560FF
:10869000E079002804D007E00022E2E70122E0E7C9
:1086A0000120E07101F08AFF80213046FEF7B0FA28
:1086B000002806D0002208213046FEF7B6FA012233
:1086C00005E0012208213046FEF7AFFA002205201E
:1086D00039460007FEF7A9FA244C284E4034A08CF6
:1086E000274F012803D01CE0E5710022EAE7254866
:1086F0006946088072B680212348FDF79DFB00285B
:1087000004D0022269462048FDF73AFC62B61FA059
:1087100001F0F2FFA58403F02FFF642002F04AFA73
:10872000FE60608C012808D110486584058003F044
:1087300023FF642002F03EFAFE60208C012806D15F
:10874000258403F019FF642002F034FAFE60074824
:10875000124A0188914202D1C088002800D1FE60EF
:10876000F8BD00009016002024010020DC0D002040
:108770000004005082000020680100200400FA0577
:1087800000ED00E0AAAA0000384A0008BDF8C8EBD6
:10879000C9FDBCB6C4A3CABD0D0A0000AA5500009D
:1087A00008B55721202000F06AF80321212000F0AD
:1087B00066F84021222000F062F80821232000F012
:1087C0005EF8AA21302000F05AF8084801210187FC
:1087D000322000F054F80221332000F050F86846AF
:1087E00000F006F80A2002F0ECF908BDDC0D0020CC
:1087F00010B501460F2000F021F8002800D001201C
:1088000010BD10B50446FFF78DFE3220FFF75DFE68
:10881000FFF7C1FEE0B2FFF758FEFFF7BCFEFFF71F
:1088200081FE3320FFF751FEFFF7B5FE0020FFF772
:108830001FFE0446FFF791FE204610BD10B50C4602
:10884000FFF7DFFF2070012010BD70B50D46044614
:10885000FFF768FE3220FFF738FEFFF79CFEE0B21C
:10886000FFF733FEFFF797FE2846FFF72EFEFFF7D0
:1088700092FEFFF772FE0A2002F0A3F970BD10B558
:10888000FFF7E3FF012010BD10B50248FEF719FB0A
:1088900010BD0000C8150020FEB50446002772B6C2
:1088A000334A01688B1804D13248C768032080041A
:1088B000074088680190C868009048698E69002B5D
:1088C00008D12C4940398B6ACD042B438B628B6ACB
:1088D000AB438B62014631433CD025492368CB42F0
:1088E00005D12449CA6803239B049A43CA602546DC
:1088F0002035002810D021680A6901231A430A6133
:10890000216848610821204600F036F8032800D18C
:10891000A873216808204860002E10D020680169E3
:10892000012211430161206886611021204600F078
:1089300023F8032800D1A8732168102048600C4850
:108940002168C14206D10B48C168032292049143B9
:108950003943C16020680169490849000161216803
:108960000198886021680098C86062B6FEBD00006A
:108970000084FFBF4010024070B506460B480D460C
:10898000002409490068FCF7B3FB7D21C900484376
:108990003168401E00D103240B682A469A4301D057
:1089A0000028F6D1204670BD204E0000780100203E
:1089B0001CB5002116480091144A01910260C16360
:1089C0001205426081600722826301220261024631
:1089D000C16020321170FF235170C2334362816243
:1089E000117301638161042241634261C161FDF73A
:1089F000FDFC084800908013019069460448FDF78B
:108A0000A5FC00210248FDF74BFC1CBD00240140E1
:108A10006C1500200200000408B50848016B012213
:108A200011430163006B01211040009000220A20D5
:108A3000FEF794FB0A20FEF785FB08BD00100240FC
:108A4000F0B587B014216846FCF7B1FB4748C26A0D
:108A500004210A43C262C26A0A400592C16A8026A2
:108A60003143C162C16A31400591C16A0124214389
:108A7000C162C16A21400591C16A02252943C162D0
:108A8000C06A22462840059005201C210007FEF7F9
:108A9000CCF8012236493748FEF7C7F8002236499C
:108AA0003448FEF7C2F89121052000220902000790
:108AB000FEF7BBF831480190002705206946029770
:108AC00000940007FDF7E8FF0C20009011200190B2
:108AD000032003900520029769460007FDF7DCFF9D
:108AE00010206A46039591C2052069460007FDF7EC
:108AF000D3FF1120019002976946039700941D4807
:108B0000FDF7CAFF1E480190694600950294194876
:108B1000FDF7C2FFE00200906946019702951548F3
:108B2000FDF7BAFF1748694691C169461148039796
:108B3000FDF7B2FF91200002694691C10520694608
:108B400000070397FDF7A8FF69460A4801970096BA
:108B50000294FDF7A1FF002201210520FEF7FEFA95
:108B60000520FEF7EFFA07B0F0BD0000001002404C
:108B70000102000000040050083000000000111045
:108B8000000021100832000010B50F4C0D48206085
:108B9000FF20053060600020A060E060206160611F
:108BA000E0610121206249026062A161A0620720A8
:108BB000E0622046FEF71FFF206801684022114353
:108BC000016010BD00300140F815002010B58AB0DA
:108BD00000240494059406940794089401211848ED
:108BE0000994009401940294890703940160092177
:108BF00084604160046113494461C160FEF7C6FFAF
:108C000001200003049004A90D48FEF7EDFF0C4875
:108C1000FFF7DCF8089408A909480994FEF78AFFD1
:108C2000602000900848019002940822694603944D
:108C30000348FFF767F80248FFF73EF80AB010BD97
:108C400050160020930400005702000000B585B0C4
:108C500014216846FCF7ABFA0E480D490160E1218A
:108C60004902416000218160C160016181610C2283
:108C7000C1614261016230214162012109038163C6
:108C80004900C163FFF738FA01F092FC05B000BD5E
:108C9000003801409016002070470000F0B585B004
:108CA0000A2002F0D9FC7D20C00002F0EFFCFF4C4E
:108CB0000025A570FE486065A07B0C2801D30B2021
:108CC000A073FC48E570FC4E00783071FB49A07938
:108CD000097840000843217D89000843F071E06A6B
:108CE000F070010A3172401CE0626079F449B0749E
:108CF0004200C81FFE38FCF741FA6079F049820053
:108D00004000801960311330121DFCF737FA2A2019
:108D1000205E002803D0EB49098A08186085607935
:108D200006214843E44EE149821922310B7AD3757A
:108D3000497A117606217172E349DC4A0978B172E9
:108D4000217F317331461339937F0B75D27F4A757A
:108D5000002213311C3002F069FD6079062148437E
:108D600000211C3002F074FD022002F0C5FCF571F8
:108D70002574E572012767732573D448FEF77CF9E3
:108D800060840646E5706079FCF7D8FCD04AD14B88
:108D9000FCF7B8FB01F0AAFE0022BB07FCF700FBC2
:108DA000FCF72CFD0006C10C881980B2F903A084E1
:108DB000884201D3401AA084C748E0632079401C50
:108DC0002071C248FEF758F92084D5E1BF48FEF76C
:108DD00053F92084C14E0BE0BC48FEF74DF980B238
:108DE0002084A18C884203D3BD4A8918884206D3C7
:108DF00000210F2002F0B0FB30422063ECD0206B4A
:108E0000411C21D040047DD58122D20100210F20B8
:108E100002F0E1FC7D20C00002F038FC002002F0EE
:108E2000EAFB0021102002F097FB4106A448490EFE
:108E3000264600226438216502F0C4FBA04864384D
:108E4000417A0729C1D101E001F0D4FC0222A549F1
:108E5000401DFCF7B7F90028B7D102F04AFD716652
:108E60003446306602F032FDF166B066F07869464D
:108E7000401CF07092486B38027A0A70407A487051
:108E800008880090F18B88427ED18B48964E8C30BA
:108E9000C08E3080884885498C30008F48838B484D
:108EA000FEF7EAF8208402F069FAFF22A16E52046C
:108EB000E06E0023891858410206080A1043410851
:108EC00049000090080E0902216760677A48636EC6
:108ED0000A30226E02F0E2FC6079E36E810076488F
:108EE000A26E0818163002F0D9FC7348636F123076
:108EF000226F02F0D3FC704808214172E07C002808
:108F000016D000E02BE16E48022276495F38FCF76C
:108F100059F900280CD168482774C771206D684939
:108F20001638C2B24E3908466274EA30FCF726F9A8
:108F300060790022800060491C3002F077FC607983
:108F4000002180001C3002F083FC009802F07DFBC1
:108F5000012002F0D1FB607202216448FDF758FE47
:108F600000287DD000215548554A017052494F488C
:108F70008C314B8E0387898E4187A06B6032E06312
:108F800010602064104600E080E0C438C27C100706
:108F9000000F032800D0A0741009E074257101208F
:108FA000424AE0729387D1872073608B5049FF302B
:108FB000C33080B2608388420BD949424018608335
:108FC00030887D21401C80B2C9003080884200D3A7
:108FD000358036887D20C000618B70434018606406
:108FE00004904448302107784348E7730088484399
:108FF000FCF789FB00900A2031464143A08B3022C8
:1090000003905043081AFCF773FB0099FCF77DF9B5
:109010007F21C905FCF7E3F8FCF7B7FB80B23549BF
:109020007F1E0880B84201D101202073E6841620FB
:10903000205EFCF76FFB06460F46208CFCF77EFB9C
:109040002E4A2F4BFCF75EFA009001910498FCF732
:1090500061FB019B009AFCF747FA32463B4600E071
:109060000BE0FCF79DF9FCF7A5FBA064039800F06A
:10907000EFFC607A002802D087E0012173E700212D
:109080000F2002F069FA0006F9D57EE0FCF794FFA4
:109090000B4A032190321154FF3A1D3A0349538E73
:1090A0000B87928E86004A8705482BE070000020CF
:1090B0003F420F00240100205012002064010020D4
:1090C000681300201C0E002034010020C815002069
:1090D000B81E85EB51B8CE3FA086010000D02724F2
:1090E000983A000048010020600100200004005070
:1090F000E70300004001002044010020F853E3A5ED
:109100009B843E40554930303018898F0180534848
:10911000A16BEC30301841605048E36E8C38301849
:109120001630A26E02F0BAFB616DA06B884207DABE
:109130004A49BC318959012902D1606500990291DF
:109140004649BC318959814216DD012914DD214689
:10915000002811DD0098C883022020700CE0324600
:1091600000210F2002F037FB6079E178401C81423A
:1091700002D0002002F03FFA208CA18C884200D25D
:1091800024E6374A89188842FAD8E07A012801D0C3
:109190000220E07202F0F2F8324A00210F2002F0C1
:1091A0001AFB2079002810D02F4909888A008918D5
:1091B000814200D22570207C002834D02B490B78C6
:1091C00048788A78022B16D02DE0E16B626D323937
:1091D00020468A420DDAC179234A491CC9B2C171BD
:1091E000128852008A42E6D20299C183022121707C
:1091F000E1E7E571DFE710280CD0C82813D21C4B3B
:10920000C91C1818FBF7BAFF03F0B6F9642001F087
:10921000D1FC19E6174D28684000000E03D1C8782C
:10922000FCF771FA28600D4D00208C352E46217810
:109230006279183607E04300EF5AF35A9F4200D094
:109240000221401CC0B29042F5D3064A2170803200
:1092500000210F2002F0BFFA05B0F0BDDC120020A3
:10926000983A000000D02724340100200414002084
:10927000DC0D00204C01002070470000F0B58BB0E1
:10928000002005900A2002F0E7F97D20C00002F0DE
:10929000FDF9BF4800218170C26ABF4C521CC262F6
:1092A000BC4A438D128A2546D21842854175214613
:1092B000133108912230473103903135204613385D
:1092C000B64F02910690B24E0F21B54871710078E9
:1092D0002071B44AB079127840001043327D920078
:1092E0001043E071B08DE070000A2072A174314625
:1092F0001E2284310898FBF741FF40222846AA49E4
:10930000FBF73CFF039902980A7AC274497A017507
:1093100009206072A5480078A072307F2073707DAC
:10932000410030468430091806980A780275497859
:10933000417576200022984902F078FA707906216A
:10934000484300211C3002F083FA022002F0D4F9D5
:1093500000210F2002F000F938423063F8D0306B62
:10936000411C18D040047DD58122D20100210F205C
:1093700002F031FA0021102002F0EEF84106864892
:10938000490E0022B43002F01DF98348B430417A0E
:10939000022902D0D4E001F02DFA02228449401DB6
:1093A000FBF710FF0028F5D179480222407D4100EB
:1093B0007748843009187848B530FBF703FF002858
:1093C000E8D102F096FA724E7166306602F07EFACB
:1093D000F166B0660598002848D1012005906E48D6
:1093E000744E8C30C08E6C49308069488C31098F46
:1093F00041837148FDF740FE6549704A0884488BF7
:10940000FF30C33080B2488390420CD9524280185A
:1094100048833088694A401C80B20B3230809042C9
:1094200001D300203080308859497D22D2004B8BF7
:109430004243D2184A64624A064613880A3EDAB2A8
:1094400036B2CA730E85002E04DA7D21C900711868
:109450004F4E31854E49521E934201D101220A736B
:10946000C88400E08DE0888B00F0F2FA4A48694633
:109470008C30428E0A80808E488047490422B53164
:10948000C81FFF38FBF77AFE4148474A407D0099E4
:10949000800011503E48FF23816EC06E5B040022A5
:1094A000C918504100060E0A0643304602F0CDF8B6
:1094B000710849000A0E0802354900264A67086704
:1094C0000846436E026E3448483802F0E7F93048E7
:1094D000C36E826E3048443802F0E0F92C48436F86
:1094E000026F2D48403802F0D9F92B490022523939
:1094F0003C2002F09BF900213C2002F0A9F9012058
:1095000002F0FAF82249487208468078401C8870B8
:1095100001210520C9030007FCF762FD1C48407AC1
:10952000002805D100210F2002F016F80006F9D519
:10953000802200210F2002F04EF915494E7002E002
:109540001349012048701248417D491CC9B2417538
:109550000F2900D2B7E60598002810D10C48194908
:10956000828B002A02D00B889A4201D90988818314
:109570001549808B0988401E4843144908800BB068
:10958000F0BD134A00210F2002F025F9D8E70000B2
:10959000700000201C0E00205012002000D0272454
:1095A0002401002064010020541400203401002014
:1095B0004801002060010020C8150020E7030000DA
:1095C00040010020300100202E0100202C0100204D
:1095D00000902724F8B532493048086002F070FA4C
:1095E000304800F0F5F9304CE0822E48801C00F045
:1095F000EFF920832B48001D00F0EAF960832C4826
:109600002A494180014640310A792A4F1206120E3A
:10961000627006D1C7800122C2870A2242870022D7
:10962000828702890A82244AC18E1170C18F6171BA
:10963000818FA171817AE1708588052165626181E0
:10964000C6883046FBF754FDA08101462846FBF74B
:109650004FFD8800081885B2164825816843FCF73D
:109660006DF8164A164BFBF7B5FFFCF7C7F8E0811B
:10967000658231463846FBF73BFD20820146C82013
:10968000FBF736FD20840120A083FCF7ADFCA0820F
:10969000E2890C490C48FDF7F3FCF8BDE9A5000888
:1096A00068000020004F0008240100202302000071
:1096B000DC0D0020E803000018000020F853E3A5AB
:1096C0009B843E40FF7F0000C8150020F0B59A4DF6
:1096D00085B001202880994FC820994C3880207A85
:1096E000401C2072C00706D0A08B411EA183022817
:1096F00001D2C820A083A08B00F0AAF90A2001F0B3
:10970000ABFF7D20C00001F0C1FF02218D48FDF7B5
:109710007FFA00283FD000208B49800009788C4ECA
:1097200049000843894909780843B07210207072D3
:109730008848C1887D20C000FBF7DAFC707386483A
:1097400084490078B07330460B308A780270C9784B
:1097500041708049421C20310B7ED370497E1171CB
:109760007C49D01C22310B7E5371497E917179491D
:1097700040310A7C0271497C417100223146172038
:1097800002F054F80021172002F062F8022001F0E4
:10979000B3FF724E03E00120BEE7FEF727FF002172
:1097A0000F2001F0D9FE30422063F6D0206B411C1F
:1097B0007ED040047DD58122D20100210F2002F00D
:1097C0000AF80021102001F0C7FE41066048490E4A
:1097D0000022B430216501F0F5FE5D4EB436707A9A
:1097E000112866D102225E49701DFBF7EBFC0028B0
:1097F0005FD1F01F027A69460A70407A4870B17AE8
:109800002980C820FBF774FC3880307BA083304669
:10981000544D2838C08E2880314649482839098F50
:1098200041835148FDF728FC80B220840390608B6F
:109830004E49FF30C33080B2608388420CD9494220
:109840004018608328884949401C80B20B31288029
:10985000884201D3002028802D887D20C000618BA4
:1098600068434018606402904148067828460A38E8
:1098700000B2E6732085002803DA7D21C900401874
:109880002085388830214843FBF73DFF07462820D4
:10989000205EFBF72DFF3946FBF737FD7F21C90519
:1098A000FBF79DFCFBF771FF314980B2088001E0B6
:1098B0003FE03CE0761EB04201D101202073E584F8
:1098C0001620205EFBF726FF074601910398FBF761
:1098D00035FF284A284BFBF715FE05460E46029831
:1098E000FBF718FF2A463346FBF7FEFD3A46019B7D
:1098F000FBF756FDFBF75EFFA06468460088E08337
:1099000013481349B430807CC73160714200084667
:109910000D465130FBF732FC60792946420017486A
:10992000FBF72CFCA08BFF2801D00320207005B092
:10993000F0BD00F05FFF0000340100204401002072
:109940007000002000040050290100202A0100209E
:1099500050120020DC0D00201800002000D0272429
:109960004801002060010020C8150020E703000026
:1099700040010020F853E3A59B843E408013002063
:1099800070B586B014216846FBF711FC01250F4E17
:10999000ED03002229463046FDF747F90120002457
:1099A000019002946946009503943046FDF774F8DF
:1099B0000320019002946946009503943046FDF718
:1099C0006BF8022001F0F6F806B070BD00040050FC
:1099D0000088704770470000F8B5044600206A46CA
:1099E0001080194D55222A70AA226A700322AA708B
:1099F000661DEE702A716971144A49008918AC71AC
:109A00002246E81DFBF7BAFB002007E029186A464A
:109A10008978128889186A461180401CB042F5DBAB
:109A2000611DA81CFCF736F901466846018029191A
:109A30000078C871684640780872214609310248AA
:109A400000F0E2FBF8BD000008150020DC0D00204E
:109A500010B51B4C228A01E0891AA183A18B914287
:109A6000FAD2228C8BB253431B18E383132902D101
:109A70004A431018E083E08B30214843642164306E
:109A80004843104960630968401A4B210901401896
:109A90002063FBF73FFE0C4A0C4BFBF79BFDFBF7EB
:109AA00089FE0B49E062884202DD4A428018E0628A
:109AB000002801DA4018E06206490968486110BDD3
:109AC00024010020B8000020F853E3A59B843E4009
:109AD000FF7F0000C8150020034A1168382389B2AF
:109AE00099430143116070470030014010B5FDF704
:109AF000A9F810BD10B59AB034216846FBF757FBA2
:109B000014210DA8FBF753FB1C2112A8FBF74FFBF8
:109B10001B4801680324E402A143C21489180160B0
:109B2000FDF728FB17480169A14301610620009059
:109B3000FF200130029001200390102004900220A9
:109B4000099040040B90000100240C900A94684690
:109B5000FDF73EFD0F200D9003200E900F94109402
:109B6000012111940DA8FDF709FC8120129003201A
:109B700080041890149412A8FDF74EFB1AB010BD83
:109B800000700040401002401048016882151143E7
:109B90000160C1680E4A1140C16001680D4A114060
:109BA00001608168490849008160016801229204CE
:109BB00091430160C168FD2212049143C1600021FC
:109BC00001610649044888607047000000100240A7
:109BD0000C40FF88F6FFF6FE0050000800ED00E0A4
:109BE00070B5026801239B07114C124D984203D0B7
:109BF000A04201D0A84203D17026B2434E6832433E
:109C0000984203D0A04201D0A84204D103231B02F2
:109C10009A43CB681A4380239A430B691A43026024
:109C20008A68C262096881620121416170BD0000D9
:109C3000000801400014014010B5CB06DB0E0121E5
:109C4000046A99408C430462016A9A40114301629C
:109C500010BD30B58468FF252D021B021343AC43B1
:109C60000B432343836030BD826870239A430A43C9
:109C700007210A438260704730B5026A52085200D9
:109C80000262026A456883697024A3439C080B68DA
:109C9000A40023430224A2438C68456014438361DB
:109CA00049684163046230BD30B5026A10239A43AB
:109CB0000262036A4568826973242402A2430C6825
:109CC00024021443202293438A68456012011A43F8
:109CD000846149688163026230BD30B5026AFF2346
:109CE00001339A430262026A4568C3697024A34340
:109CF0009C080B68A400234301246402A2438C68DF
:109D0000456024021443C3614968C163046230BDE5
:109D100030B5026A01231B039A430262036A456855
:109D2000C26973242402A2430C6824021443012252
:109D3000520393438A68456012031A43C461496819
:109D40000164026230BD30B5036A046A64086400CD
:109D500004628469F025AC43120122430A24A34320
:109D60000B438261036230BD30B5036A1024A34304
:109D700003628469036A0F252D031203AC43224357
:109D8000A024A343090119438261016230BD000090
:109D9000F8B5102605252D07AE62AF20800000F033
:109DA00010FFFCF7BDF9364834490068FBF770FA3C
:109DB000FBF7D2FC334C6085AE6101F0E1FB324F22
:109DC000324EA0650EE001F0DBFBA065FEF70EFC55
:109DD000606B411C6163142804D92DA000F08CFC39
:109DE0002F48C760A06DB042EDD100266663207891
:109DF0000127FF03030000F0B8FC05040C192D3007
:109E00003200012239462846FCF70FFFFFF75EFCBF
:109E100006E0012239462846FCF707FFFFF72EFA35
:109E2000002239462846FCF700FF18E0A07A0122FC
:109E3000401EA07239462846FCF7F7FEFCF7F0F802
:109E4000002239462846FCF7F0FEA07A002806D109
:109E5000267004E0FEF722FF01E0FFF70FFA02216F
:109E60001048FCF7D5FE002805D000200E490870E8
:109E700001F06CFAF8BD0120F8E700000000C842CC
:109E800000000020700000200400FA053001CADE46
:109E90004457204944204552524F522E0D0A00008B
:109EA00000ED00E0000400506401002010B5818C3A
:109EB000C90707D001684A6801235B049A43836A93
:109EC0001A434A60818C890707D501684A680123D3
:109ED0001B049A43C36A1A434A60818C490707D519
:109EE00001684A6801239B049A43036B1A434A6042
:109EF000818C090707D501684A680123DB039A436F
:109F0000436B1A434A60818CC90607D50268916881
:109F100001231B039943836B19439160818C89064C
:109F200007D501688A6801235B039A43C36B1A4310
:109F30008A60818C490612D503685A680121090597
:109F4000046C8A4322435A60026C8A4207D1026839
:109F5000516803235B059943436C19435160818C1D
:109F6000090607D501684A680123DB04806C9A431F
:109F700002434A6010BD0000F8B504460026803058
:109F80000660FCF759FE054620680068124F00077E
:109F900009D501212B46002249052046009700F0F3
:109FA000ABFA00280DD12068006840070BD50121CD
:109FB0002B46002289052046009700F09DFA0028D4
:109FC00001D00320F8BD2020A067E067266660343A
:109FD00026750020F8BD0000FFFFFF01F8B5184C02
:109FE000C826E078002829D16079002826D10120F0
:109FF0006071144D686B002700281ED0686BC82163
:10A00000081A15E01048E168405C616988470F480C
:10A010000A21008848430E490880E068401CE0603F
:10A02000E068C82800DBE760696BC820401A761E2C
:10A03000E168814201D0002EE4DC6771F8BD0000C8
:10A040005400002000000240140D002034010020C4
:10A050004601002070B5224CE07800283FD12079DD
:10A0600000283CD1012020711E4EF169002509060F
:10A07000002933DA2156625791420AD1F06940062D
:10A080002CD5A079002829D0A5712089401C2081D9
:10A0900024E0A179002903D1A0710A2000F091FDEC
:10A0A00000202056CC2148430F494218206912183D
:10A0B0001279B262401C00222061A256CC235A437E
:10A0C000895881420ADC25612078401C2070207864
:10A0D0000E2800D12570A078401CA070257170BD9D
:10A0E0005400002000380140EC01002010B5806AC7
:10A0F0000022014640314A834A82FDF7EBFE10BD43
:10A1000070B5846AA06FE56F21688968002609062A
:10A11000002906DA212804D152200653204600F0F7
:10A120006BF820688068400606D5222D04D15A209D
:10A130000653204600F047F8204680300168102280
:10A14000114301602046FDF7C5FE70BD10B5014604
:10A150000968806A096889061CD400225A210A52BB
:10A1600001680A68FF2301339A430A6001688A681C
:10A17000520852008A6001688A6840239A438A60C4
:10A180002021C167016E012904D101680A681023EA
:10A190009A430A60016E012902D0FEF77DF810BDD6
:10A1A0005821095AFDF794FE10BD10B5806A016E62
:10A1B000012902D0FEF771F810BD5821095A49084B
:10A1C000FDF786FE10BD01680A68FF2321339A431C
:10A1D0000A6001688A68520852008A60016E01298B
:10A1E00004D101680A6810239A430A602021C167DC
:10A1F000002101664166704701680A68C0239A43DE
:10A200000A6020218167704770B5164CE278002AF9
:10A210000CD12279002A09D10122E2700025C82937
:10A2200003DC0222A256002A01DCE57070BD012386
:10A23000E356CC2253430C4AD1500123E356CC269B
:10A2400073439B180A460146181DFAF797FF60787A
:10A25000401C607060780E2800D16570A078401EA8
:10A26000A070E2E754000020EC010020F8B504469D
:10A27000016880682369E6691843636900253343F0
:10A280001843724A0B68724E334003430B602168D7
:10A29000486803231B039843E36818434860216818
:10A2A000A069914201D0236A18438B680B263602BD
:10A2B000B34303438B606749236867488B420CD1E3
:10A2C000C0688007800F06D0012839D0022835D019
:10A2D000032821D11EE001271FE060498B420AD1EB
:10A2E000C0680C21084027D0042829D0082825D090
:10A2F0000C2811D10EE093420ED1C16803208002D8
:10A30000014019D001208002091A19D0091A15D06C
:10A31000814201D1082700E010274F4950484039B9
:10A320008600934232D1002F0CD0022F0DD0042F83
:10A3300010D0082F7FD126E00027EEE70227ECE7B8
:10A340000427EAE7FDF7E8F806E00968C90605D43E
:10A35000304603E0FDF700F9002872D06268510032
:10A360005118814267D81103814264D3010E06025D
:10A370005008002330185941FAF7D0FE0321090292
:10A38000411A384A55E00120C003E7E70122E3699A
:10A39000D20393422BD13B0000F0E7F90906090CE8
:10A3A0004D114D4D4D274D00FDF7B6F809E0FDF775
:10A3B000C3F806E00968C90605D4304603E0FDF796
:10A3C000CBF800283DD0616840004A088018FAF7B1
:10A3D0008FFE80B20146244A103991422BD8511C7D
:10A3E00001400007400F084329E01046EBE73B001F
:10A3F00000F0BBF90906090C2112212121232100BB
:10A40000FDF78AF80AE0FDF797F807E00968C90642
:10A4100006D4304604E00EE0FDF79EF8002810D088
:10A4200061684A081018FAF763FE80B201460E4AC6
:10A430001039914203D9012503E01046F0E7216865
:10A44000C86000206066A0662846F8BD004800404D
:10A45000F369FFEF00380140401002400044004023
:10A4600000093D00FFFC0F00EFFF0000F8B50446B7
:10A470004165403000262746028380373E60222017
:10A48000E0672546206F603500281CD01749C1625F
:10A49000216F17480863216F16484863206F866351
:10A4A000236F606D9C461346216802466046243146
:10A4B000FCF71AFA002806D0102038602E752020EC
:10A4C000A0670120F8BD2E7520680168FF220132C7
:10A4D0001143016020688168012211438160206876
:10A4E00081684022114381600020F8BD4DA1000821
:10A4F000ABA1000801A10008FFB581B005460F46D9
:10A50000044660350A9E39E0701C37D0FCF794FB96
:10A510000499401AB04222D8002E20D02068016849
:10A5200049072BD5C069C043000527D40120216805
:10A53000C002086220680168FF22A13291430160D5
:10A54000206881684908490081602020A067E06791
:10A550008034206000202875032005B0F0BD2068FD
:10A560000168FF22A1329143016020688168490897
:10A57000490081602020A067E067EBE72068C1699F
:10A580003846884305D0002103988142BCD0002082
:10A59000E3E70121F8E7000010B50449102009683D
:10A5A00008620248FDF798FC10BD000090160020DC
:10A5B00001490D20887070475400002010B50748ED
:10A5C0000A22018A51434184FEF726FAFEF73EFB38
:10A5D000C82203490348FDF72FFE10BD24010020C7
:10A5E000140D002090160020F8B53E4C0023217871
:10A5F0003D4A1D46082910D0072947D0062950D0CA
:10A60000052952D0042953D0032954D0002956D00B
:10A61000012958D002295AD05BE0A17800264A1FB0
:10A6200004E0314FBF5DFB189BB2761C9642F8DB0D
:10A63000667927799A195118E3786278C9188918C8
:10A64000C9194018C0430006000E1AD1012E14D0BB
:10A65000022E16D125482449C018FAF78FFD01F0C3
:10A660008BFF642000F0A6FABFF34F8F21492048EA
:10A67000C860BFF34F8F00BFFDE759081046FFF7D2
:10A68000ABF92570E570A570A571F8BDA17950549E
:10A69000491CC8B2A071A178491F8842F5D1082091
:10A6A00001E0607007202070F8BDE0700620FAE736
:10A6B00060710520F7E7A070E5700420F3E75528E6
:10A6C00007D10120EFE7AA2803D10220EBE70328F6
:10A6D00003D02570E570A570F8BD032020702071AF
:10A6E000F8BD00001C010020A4140020DC0D002097
:10A6F0000400FA0500ED00E010B5024A024900F03E
:10A70000E5F910BDB5B800087C0100202021020C3D
:10A7100001D010211046020A01D010460839020962
:10A7200001D01046091F820801D01046891E420838
:10A7300001D0881E7047081A7047F8B5040C8BB218
:10A74000264682B25E430D0C1046370C5843360441
:10A7500080190021794116466E43370C3604801962
:10A76000794126466E438919F8BD30B47446641E9B
:10A770002578641CAB4200D21D46635D5B00E31884
:10A7800030BC18474900CA020243100000D0042020
:10A790004A0D01D001221043044A490D914201D1D2
:10A7A00002210843012800D105207047FF0700005F
:10A7B0008307FF22DB0E9A408907090E9940002883
:10A7C00008DB830809489B001B181868904308435E
:10A7D000186070470007000F0838830804489B0082
:10A7E0001B18D86990430843D861704700E400E023
:10A7F00000ED00E0BFF34F8F04490348C860BFF38A
:10A800004F8F00BFFDE700000400FA0500ED00E0F7
:10A81000F8B504464F1EC8000838211815461E46D4
:10A82000086849683A4606239A4310D02A463346B8
:10A83000FAF768FE3A46D200083AA3181A687F1E53
:10A840005B68FAF7ADFD06223B469343EED1022F3B
:10A8500023D0042F11D0062F2FD12A463346FAF7E2
:10A8600051FEE36AA26AFAF79BFD2A463346FAF7DD
:10A8700049FE636A226AFAF793FD2A463346FAF7DD
:10A8800041FEE369A269FAF78BFD2A463346FAF7DF
:10A8900039FE63692269FAF783FD2A463346FAF7DF
:10A8A00031FEE368A268FAF77BFD2A463346FAF7E1
:10A8B00029FE63682268FAF773FDF8BD002210B51F
:10A8C000134610460149FAF785FE10BD0000F03F1F
:10A8D00010B5FAF765FD10BD002210B513461046FD
:10A8E0001146FAF777FE10BD10B50721024A002085
:10A8F0000907FAF7E7FE10BD01030000034A10B58F
:10A9000000201107FAF7DEFE10BD000001FDFFFF79
:10A9100002E008C8121F08C1002AFAD17047704728
:10A92000002001E001C1121F002AFBD17047000086
:10A9300001490860704700008001002008B500212F
:10A94000684601706B46012202212C2000F052FF64
:10A950000221684601706B4601222C2000F04AFF5C
:10A9600008BD000038B504466D20694608706B4686
:10A97000012207492E2000F03DFF0649002C01D09E
:10A98000054A00E0054A2E2000F01AFF38BD0000FD
:10A990000608000006180000070600000716000061
:10A9A00038B504466B4602220021362000F0EEFD49
:10A9B000B3212300FFF7D9FE0E0F08153A3A3A3AB1
:10A9C0001C273A3A2F34483A0021684601704078F3
:10A9D0004108490014E06946087880088000401C5E
:10A9E00004E06946087880088000801C08701DE03B
:10A9F000684602780A40483202704178802001435C
:10AA00006846417012E0684602780A400270407859
:10AA10004106490EF4E7694648780221084303E0FD
:10AA200069464878FD210840694648706B46012216
:10AA30000021362000F0DEFE012200AB1146362058
:10AA4000013300F0D7FE38BD69460878CF210840B1
:10AA500069462030CAE708B50321684641700121E4
:10AA600001706B4602220021362000F0C3FE012255
:10AA7000D20306212D2000F0A3FE012000F09AF859
:10AA80000120FFF78DFF08BD08B5020A69464A702C
:10AA900008706B46022204212D2000F0ABFE03203B
:10AAA000694608706B46012206212D2000F0A2FEA7
:10AAB0000020694608706B46012206212D2000F017
:10AAC00099FE0A212D2000F047FD08BDF8B5164675
:10AAD0000F460446002503E03946B047641C6D1C50
:10AAE00020780028F8D12846F8BD0000F8B54A00C3
:10AAF0002B4B520DD6182B4A0C460546142E2BDA3A
:10AB0000002E12DA284BFAF74BFC00221346FAF714
:10AB1000BBFE40D2002C03DA0124E40700253AE012
:10AB20002046284337D0214C14E0214F0B46F740F4
:10AB30003B402B4331D01C4BFAF732FC002213462A
:10AB4000FAF7A2FE27D2002C03DD01200005F04019
:10AB50000419BC4300251EE0332E1EDC33460027BB
:10AB6000143BFF43DF40384217D00F4BFAF7C2FCCB
:10AB700000221346FAF788FE0DD2002C0ADD142EAF
:10AB80000CD03420811B012088404019A84200D2FB
:10AB9000641C0546BD4321462846F8BD641CF9E700
:10ABA00001FCFFFF9C7500883CE4377E0000F03F0D
:10ABB000FFFF0F007D2110B5C900484300F001F8E8
:10ABC00010BD002140E000BF00BF00BF00BF00BFBC
:10ABD00000BF00BF00BF00BF00BF00BF00BF00BF7D
:10ABE00000BF00BF00BF00BF00BF00BF00BF00BF6D
:10ABF00000BF00BF00BF00BF00BF00BF00BF00BF5D
:10AC000000BF00BF00BF00BF00BF00BF00BF00BF4C
:10AC100000BF00BF00BF00BF00BF00BF00BF00BF3C
:10AC200000BF00BF00BF00BF00BF00BF00BF00BF2C
:10AC300000BF00BF00BF00BF00BF00BF00BF00BF1C
:10AC400000BF00BF00BF491C8142BCD37047FFB5A5
:10AC500081B01E460F46040026D00B99039801438D
:10AC6000A06A3943826807209047002818DB0A99B8
:10AC7000A06A3143826806209047002810DB2546F1
:10AC80002035A979032F01D908200143032E01D9CA
:10AC900004200143A06A826809209047002806DA50
:10ACA0000120C04305B0F0BD0020C043FAE738469C
:10ACB00000F000F92060304600F0FCF860600A986F
:10ACC00068700398A870EF702E710B98687100205F
:10ACD000E8E70000F7B50446002090B0009001902E
:10ACE000002C05D06A46062101F080FC062803DA14
:10ACF0000020C04313B0F0BD6846407801026846AA
:10AD0000007800040918684680780818FAF716FDDC
:10AD1000054668460391007901026846C078000440
:10AD20000918684640790818FAF708FD0322064614
:10AD30000F4692075C4BFAF7A7FD07D200225B4B48
:10AD400030463946FAF7D0FB06460F4603229207F3
:10AD5000554B28460399FAF797FD07D20022534B2B
:10AD600028460399FAF7C0FB054603912068FAF7D5
:10AD7000E5FC02460B4630463946FAF72BFC0746FF
:10AD80000A200791205EFAF7C5FC3A46079BFAF7BE
:10AD9000B9FB064608200991205EFAF7A9FC0021BC
:10ADA000C943FAF7F0FAFAF747FD3246099BFAF77A
:10ADB000F7FA069108906068FAF7C0FC02460B4665
:10ADC00028460399FAF706FC05461A200E46205E2F
:10ADD000FAF7A0FC2A463346FAF794FB0C90099147
:10ADE0001620205EFAF796FC099B0C9AFAF7D8FA1F
:10ADF00005910A902A46334638460799FAF782FBAE
:10AE0000059B0A9AFAF77EFB05910A901420205EB2
:10AE1000FAF780FC3A46079BFAF774FB07461C20BA
:10AE20000791205EFAF776FC2A463346FAF76AFB6A
:10AE30000E900B911820205EFAF76CFC0B9B0E9A7B
:10AE4000FAF7AEFA2A463346FAF75CFB0B910E90FE
:10AE50002069FAF75FFC0B9B0E9AFAF7A1FA2A46D3
:10AE60003346FAF74FFB05460E46E068FAF752FC08
:10AE70002A463346FAF794FA3A46079BFAF790FACD
:10AE8000059B0A9AFAF78CFA01229207084BFAF707
:10AE900039FB02460B46129C0898069903C4119888
:10AEA0000CC0002026E70000FFFF5F41000070415A
:10AEB000E17A843F00B50121C9040300FFF755FC86
:10AEC000081A05080B0E1114171A0320C00400BD40
:10AED0000720C00400BD0F20C00400BD1F20400398
:10AEE00000BD3F20400300BD7F20400300BDFF2088
:10AEF000400300BD084600BDFEB5264F0D460400C8
:10AF00000FD0002D0DD0264600202036B071F071F4
:10AF100029680D208847002801DA7800FEBD102836
:10AF200001D03846FEBDA562E968002901D028207D
:10AF30008847204600F030F80028F3DBA06AA521FE
:10AF400082680E209047A06A962182680F20904761
:10AF5000A06A0221826862209047A06A002182686C
:10AF60000E209047A06A002182680F2090477179D7
:10AF70003020019100900623202201212046FFF776
:10AF800066FE0028CEDB204600F0AEF80028C9DBC4
:10AF90000020FEBDFFFFFFFF10B586B00446142160
:10AFA0006846FAF704F9002C7ED0A06A12214368A3
:10AFB0006A4610209847122877D168460078012207
:10AFC00001016846407812030009081843492081AE
:10AFD000884201DD801A2081684683784078000726
:10AFE000000D18186081884201DD801A6081684672
:10AFF0000079012201016846C07812050003091892
:10B0000068464079000908183549E060884201DD4A
:10B01000801AE060684640790007030B6846807933
:10B0200000021B186846C07918182061884201DDAB
:10B03000801A20616846417A007A0002081802B23C
:10B04000284801210904A282824201DD521AA2820B
:10B050006A46D37A927A12029A1812B2E282824235
:10B0600001DD521AE2826A46537B127B12029A1861
:10B0700012B22283824201DD521A22836A46D37BB6
:10B08000927B12029A1812B26283824201DD521A36
:10B0900062836A46537C127C12029A1812B2A2830F
:10B0A000824204DD501A01E00BE008E0A083A06AB0
:10B0B000016828208847002806DA0120C04306B02E
:10B0C00010BD0020C043FAE7C011C007203400289B
:10B0D00000D0802060710020F1E70000FF07000031
:10B0E000FFFF0700FF7F000010B5040009D0A06A31
:10B0F0000721826808209047002805DA0120C04314
:10B1000010BD0020C04310BD072020342070002057
:10B1100010BD0000FEB5044600200190009060794B
:10B12000734940000E5A61782578491E7148CFB2A4
:10B130000163042D77D0072D75D00021029121786D
:10B1400001736C49E379012292058969002B6CD067
:10B15000914381616748217A4173217A8269890725
:10B16000890B0A4382610021042000F034FB32463F
:10B1700061492E2000F024FB3846FFF7F3FB5F4EB9
:10B180000522705D810040185D49431807212B207E
:10B1900000F030FB5B49029801220B180B2128209C
:10B1A00000F028FB705D584980000A580C212820C7
:10B1B00000F011FBE079554980004018A179490061
:10B1C000425A0221272000F0FBFA51487E00825BA0
:10B1D0000421272000F0F4FAE079002829D0A07893
:10B1E00004282CD028206946087220220621272016
:10B1F00000F0E6FA02AB01222621272000F0FAFA3D
:10B20000444938014018E178890042580821272034
:10B2100000F0E1FAA17A601C627A0902114313D0AE
:10B2200016E000E001E0012188E71143F6088161A2
:10B2300090E764220621272000F0C2FAE0E7102000
:10B24000694608720246D1E733490172090A417220
:10B25000417A007A0A0202432021272000F0B0FA46
:10B260002E4F0C2123203A6800F0B5FAF01982889D
:10B270000421232000F0A4FAA07900280BD0E07963
:10B280002749012243180021212000F0B3FA0320AE
:10B290000190012000902A07120F100102436078EC
:10B2A00000218007000B024301980005024300982B
:10B2B000400402432079C006400902436079C00679
:10B2C00002431F2000F087FAA07861780123084329
:10B2D00002040848DB030261E179490319430A4388
:10B2E00002610021082000F076FA0020FEBD000077
:10B2F00020C70008B001002004280000C8C60008CC
:10B300002400002042000020D0C60008F0C600083B
:10B31000FCC6000800C7000841100000E8C600088D
:10B320004400002038B50C4607498A8B00210243AF
:10B330002C2000F045FA684604706B460122062175
:10B340002C2000F057FA38BDB001002010B5FFF7EF
:10B35000F5FA10BD10B504460421362000F0FCF8C3
:10B360000121C902002C01D0084300E088430246B5
:10B370000421362000F02FFA10BD000038B540201F
:10B380006946087000210E2000F0E6F8044600220D
:10B3900011460E2000F01FFA6B46012200210D20FD
:10B3A00000F028FA074A00210F2000F014FA00F0FC
:10B3B000EDF9224600210E2000F00DFA024800218E
:10B3C000017338BDF8FF2724D0010020FEB50546E3
:10B3D000042069460870514C0020607521462031D8
:10B3E000206348710873A0836063A06300F0C8F80D
:10B3F0004B4E206002E000F0C3F82060B042FAD16A
:10B400000020FFF7CDFA00F0BBF8464E2060307800
:10B41000242801D9243806E00621F9F769FE06221E
:10B42000101A40010843020601040A4301020A43BC
:10B430000243B260706000211E2000F0CCF900F0E1
:10B440009FF820606B4601220021242000F0D2F9F1
:10B450001E20FFF719FB86B2300AA0730420FFF705
:10B4600013FB074600F08CF820603806000E0DD064
:10B4700002206946087101AB012212212D2000F043
:10B48000B9F9A08B012109030843A08300F078F8E3
:10B4900020600620FFF7F8FA60600720FFF7F4FA53
:10B4A000A060F006C00E207501D110202075C0B23A
:10B4B00000F0DCF9E80707D0FFF7CDFAA08B0121F7
:10B4C000C9020843A0830AE00521362000F02EF8C7
:10B4D0001549084002460521362000F071F9012087
:10B4E000FFF75EFA0021042000F036F8A061002189
:10B4F000262000F031F81521890308430246002177
:10B50000262000F068F900222621362000F058F9A4
:10B5100000F036F820600020FEBD0000B0010020E1
:10B520003001CADE18000020FFFD000038B5094CCC
:10B5300089B280B26B46022200F028F8002806D1BA
:10B5400068464078010268460078081884B22046B0
:10B5500038BD0000FFFF000038B50024E44389B285
:10B5600080B26B46042200F011F8002806D10321B6
:10B570006846435C2202D418491EFAD5204638BDDD
:10B5800010B500210846FFF7E7FF10BD38B50029C8
:10B5900009D0402420436C462070C8B27F2906D8C9
:10B5A000607002200AE069460870012006E08024ED
:10B5B00020436C466070C809A0700320694600F003
:10B5C000B5FF38BD10B5144603460A462146112082
:10B5D000FFF7DCFF10BD10B5034605220021152042
:10B5E000FFF7D4FF10BD10B5034605220021172038
:10B5F000FFF7CCFF10BD38B505460020694608703E
:10B6000000F0C4F8FF2401342246002D01D00322AB
:10B61000120200210D2000F0D3F8002D13D06B464C
:10B62000012203210F20FFF7B1FF684600780007D1
:10B6300009D5FFF7A3FE224600210D2000F0C0F837
:10B640000020C04338BD002038BD10B5024601219E
:10B650000A2000F0C0F810BD10B5044600211A20E1
:10B66000FFF77AFF000D22030005120B02430021B1
:10B670001A2000F0B0F810BD10B5024602492E2085
:10B6800000F09EF810BD000004180000F8B5054653
:10B690006B46012203210420FFF778FF0126114C9D
:10B6A0003607002D0DD02A4600210C2000F088F826
:10B6B000694608781021084369460870A06930433C
:10B6C00007E069460878EF21084069460870A069DC
:10B6D000B0430B46A06101220321042000F08AF848
:10B6E000F8BD0000B001002010B50246002118206E
:10B6F00000F066F810BD0000F8B507460025684662
:10B700000570B807204C2E4600280ADA80206946CA
:10B7100008706B46012200210D2000F06BF801201B
:10B720002073F8076946087821D006210843694646
:10B7300008706B46012200210D2000F05BF8032108
:10B740000F20FFF7F3FE8121C900084219D04020E5
:10B75000694608706B46012200210D2000F04AF86E
:10B760000020FFF7F7FD00252673ED4309E00221D5
:10B770000843694608706B46012200210D2000F045
:10B7800039F82846F8BD0000D00100201CB56B46F2
:10B79000012203210F20FFF7F9FE684600784022BE
:10B7A000C1091040C9014000814208D0012069460A
:10B7B0000871024601AB03210D2000F01BF81CBDEF
:10B7C00008B56B461A70120A5A7089B280B202220A
:10B7D00000F010F808BD38B500236C46E254120A98
:10B7E0005B1C042BFADB89B280B22346042200F0F2
:10B7F00001F838BD38B58024002909D0C025284378
:10B800006D462870C8B27F2907D86870022009E009
:10B81000204369460870012004E020436870C8098D
:10B82000A8700320694600F02BFF38BD10B5144600
:10B83000012312189B029A4202D90020C04310BD76
:10B840000B46821E21460920FFF7D4FF002010BDC1
:10B8500010B5054A8905126901430A4300210820F1
:10B86000FFF7B9FF002010BDB001002038B5044635
:10B870006B4601220E212B20FFF788FE68460078D8
:10B88000E10640094001C90E0143684601706B465C
:10B8900001220E212B20FFF7ADFF38BD10B500218E
:10B8A00042541C06120A22431B0A491C0429F7DBD6
:10B8B00010BD000013B501231A4669460248FCF783
:10B8C000EDFC00981CBD0000901600207CB5002403
:10B8D00025466846FFF77FFE04206946220E2D02AA
:10B8E000154322020C5C1443401EF7D5204629461E
:10B8F0007CBD7CB5002425466846FFF774FE042015
:10B900006946220E2D02154322020C5C1443401E90
:10B91000F7D5204629467CBDFBF79CF9FEF7EAF8EF
:10B92000FDF78EF840494148002522C00560856139
:10B93000C5613F490562C1600838FBF727FBFDF789
:10B940006BF8FDF783F9FDF71FF9FDF731F80526D0
:10B9500001223607D1033046FBF767F9FDF73AFEBF
:10B96000FCF71EFFFAF7F6F9FAF7C4F9FCF718FD31
:10B970000721B015FFF7D6FCFFF7E8FC2D4C0A2194
:10B98000208A01224843608411033046FBF74DF9B9
:10B990002648C8222849C830FCF74EFC274F284EBD
:10B9A000207900283DD0607800283AD0FEF7A2F830
:10B9B000257120780F280AD9012211033046FBF7A0
:10B9C00034F9FEF7E5F900220121090309E001221B
:10B9D00051033046FBF729F9FEF7DAF9002201217D
:10B9E00049033046FBF721F9FCF700FE608C002884
:10B9F00001D0401E60841348618C00780843CFD189
:10BA00003878002801D00328CAD10121C902304664
:10BA1000FBF7FEF80028C3D101210846FBF7CAFB5B
:10BA2000BEE7FCF7E3FDBBE7007C0040C815002043
:10BA3000FFFF000024010020140D002082000020E0
:10BA4000000400505A00002010B586B01748FBF7DC
:10BA500020FA14216846F9F7AAFB15480090032044
:10BA6000019000200290052069460007FBF714F8BA
:10BA700069461048FBF710F869460F48FBF70CF8C9
:10BA800001210846FBF796FBFF2401342046FBF713
:10BA900069FB0A4908680422104308602046FBF746
:10BAA00071FBFBF777FB06B010BD0000C815002046
:10BAB000FFFF00000004005000080050007000402C
:10BAC00010B50122920217491748FAF7CFF9154825
:10BAD000164902888A4223D0018004218180FF21F7
:10BAE000F531C1800A21018100211E224181D2430A
:10BAF00082810122C28181834323C386022303877B
:10BB0000782343878287C28702464032118451845A
:10BB10009184C183918014238382118200F02CFDD3
:10BB200010BD0000DC0D002000FC0008AA5500003C
:10BB3000F0B51FB496B084460C460246199D18987D
:10BB40000390490068006300490840080193002AF7
:10BB500001D0012600E000269E19FE4BF6185B106E
:10BB60009E422BD36E00039F0296002F00D0012728
:10BB7000F719F84EF84BBE199E421FD3039E034699
:10BB8000F64F334309D03B469C4201D1002A04D0F2
:10BB9000019B002A05D0012604E0002039461BB095
:10BBA000F0BD00269E19EE4B9E4207D8039F029ED1
:10BBB000002F00D00127F6199E4207D92B46604678
:10BBC0002146189AFEF784FE1BB0F0BD0023002C1E
:10BBD00029DAE44EB04226DAE34EB04201DB02231A
:10BBE00021E0DE4EB0421EDBE04E070DBE19142EE2
:10BBF00009DD3427BF1B039EFE400196BE40039F14
:10BC0000BE420BD00FE0039F002F0CD11427BF1BA7
:10BC10000646FE400196BE40864204D1019BDE07E7
:10BC2000F60F02239B1B0E46164318D1002D16DA81
:10BC3000002C03D0022B01D0012B06D00220FEF7EE
:10BC400077FEFEF73BFE1BB0F0BD0220FEF770FE54
:10BC5000FEF734FE0122D20751401BB0F0BD039E17
:10BC6000002E61D1BF4EB04220D1C148844201D1E3
:10BC7000002A08D0B948814209DB002D10DB189852
:10BC800029461BB0F0BD0020B4491BB0F0BD002D0B
:10BC900006DA01222946D207189851401BB0F0BDA0
:10BCA000B4497944086849681BB0F0BDAB4FB8424D
:10BCB00025D1002D1FDA002904D0B14212D1002A6B
:10BCC00009D018E0002A72D1A649E20F0020D2075D
:10BCD00011431BB0F0BD0020E20F0146D207114313
:10BCE0001BB0F0BDB14206DA234600203946F9F711
:10BCF00071FC1BB0F0BD104621461BB0F0BDB14237
:10BD000012DA0126B607B54203D12346104619467A
:10BD1000FEE3994EB54207D1261E05DB104631469B
:10BD200000F040FC1BB0F0BD67007F081646002AFB
:10BD300040D100290AD08B4A914229D1002C0EDD36
:10BD4000002D1CDB002011461BB0F0BD022B16D0CD
:10BD5000002C14D0012B12D1002C14DB0FE0002C8E
:10BD600028DA002D09DB012B03D000207D491BB010
:10BD7000F0BD002081491BB0F0BD012B03D0002095
:10BD800001461BB0F0BD00200121C9071BB0F0BD6A
:10BD9000724A91420ED1002C01DA002B17D0022BEF
:10BDA00006D00020C043F9F7B5FC1BB0F0BD90E20F
:10BDB0000120F8E7E217521C94461A4307D00022EC
:10BDC0000892664C62465B1E1A4307D009E00120C8
:10BDD000FEF7AEFDFEF780FD1BB0F0BD0022644C07
:10BDE0000892674A90427DDD664B674A98421FDDA4
:10BDF000914202DC002D05DB4DE05848814217DB03
:10BE0000002D48DD0220FEF793FDFEF76DFD05468F
:10BE10000E460022534B21460898F9F773FB08465B
:10BE200071004908C00FC007014328461BB0F0BD90
:10BE3000914215DA002D2EDA0220FEF779FDFEF789
:10BE400053FD05460E460022464B21460898F9F759
:10BE500059FB72005208C80FC0070243114617E091
:10BE60003E4B994223DD002D15DD0220FEF760FDDB
:10BE7000FEF73AFD05460E4600223A4B2146089849
:10BE8000F9F740FB084671004908C00FC00701439D
:10BE900028461BB0F0BD0220FEF74AFDFEF72EFD3E
:10BEA00049004908E20FD20711431BB0F0BD002240
:10BEB00030463946F9F718FB012205460E46D243B3
:10BEC000F9F700FC314A324BF9F714FB2A463346A6
:10BED000F9F718FB0022284BF9F70CFB07462A4616
:10BEE000334600E064E0039110461946F9F70AFB77
:10BEF0003A46039BF9F706FB0746032209915207CE
:10BF0000244B28463146F9F7FDFA07910C90224A56
:10BF1000204B38460999F9F7F5FA074601911F4A6F
:10BF20001F4B28463146F9F7EDFA3A46019BF9F7DF
:10BF3000DBFA07460B460246099107990C98F9F778
:10BF40002FFA00250E462846079B0C9AF9F7CCFAE3
:10BF50003A4627E0FFFF1F00FFFF0F000000F03F01
:10BF60000000E0FF0000F07F0000404301FCFFFF05
:10BF70000000F0BF5A0B00000000E03F0000F0FF9F
:10BF80000000E0410000F043FFFFEF3F55555555DD
:10BF90005555D53F4715F73FFE822B6544DF5DF8C9
:10BFA0000BAE543E099BF9F7A5FA02460B4652E147
:10BFB000012500202D05A94207DA352230463946F1
:10BFC000F9F780FB06463420C0430A151218FE48D4
:10BFD000101803900803FD49000B01430F46FC496C
:10BFE000884201DC002003E0FA49884202DA01209D
:10BFF000119005E0002011900398401C7F1B0390D6
:10C0000011980597C200F4480F927844801843684D
:10C010000268394630460D930292F9F765FA0791A6
:10C020000C9030460D9B029A0599F9F7B9F9024632
:10C030000B460020E549F9F7CDFA09910490079BDA
:10C040000C9AF9F75FFA129000201090E3480D4621
:10C05000784400680E90012178104907084311992F
:10C060000D9B890440180121C90447183946029ADA
:10C070000E98F9F739FA3246059BF9F73BFA024672
:10C080000B4629461098F9F73DFA064602913B46C1
:10C0900029460E9A1098F9F735FA079B0C9AF9F78A
:10C0A00029FA3246029BF9F71FFA099B049AF9F71D
:10C0B00029FA0591129A0A902B4610461946F9F76B
:10C0C00021FA06460246C6480F460B46062178442A
:10C0D000FEF79EFB32463B460091049010461946FF
:10C0E000F9F710FA009B049AF9F70CFA06460F4686
:10C0F0002B461946129A1098F9F752F9059B0A9A9D
:10C10000F9F700FA32463B46F9F74AF9109A0791D7
:10C1100004902B4610461946F9F7F4F9B14E002267
:10C12000334609910290F9F73BF9079B049AF9F716
:10C1300037F900200746024633460091F9F7D4F953
:10C14000099B029AF9F7D0F9079B049AF9F7D2F9FB
:10C1500006460D913A462946009B1098F9F7D2F908
:10C1600007910C902B463046129A0D99F9F7CAF9AF
:10C1700005460E463A46009B05990A98F9F7C2F91A
:10C1800033462A46F9F70CF902460B460746099151
:10C1900007990C98F9F704F900250E462846079BE5
:10C1A0000C9AF9F7A1F93A46099BF9F7A3F9074662
:10C1B0000722099152078C4B31462846F9F7A2F91C
:10C1C00007910090894A884B38460999F9F79AF9FE
:10C1D00007460191864A874B31462846F9F792F97E
:10C1E0003A46019BF9F7DCF8834B7B440F9A9B1886
:10C1F0001A685B68F9F7D4F8029009910398F9F787
:10C2000089FA05910490099B029A07990098F9F719
:10C21000C7F87A4B7B440F9A9B181A685B681746DD
:10C220000393F9F7BDF8059B049AF9F7B9F80E46A0
:10C230002846059B049AF9F757F93A46039BF9F704
:10C2400053F9079B009AF9F74FF9099B029AF9F7FE
:10C2500051F902460B46199900200C900F46189888
:10C26000F9F750F9029104903B460C9A19991898E5
:10C27000F9F73AF92A463346F9F744F9029B049A4A
:10C28000F9F78EF809910E902A46334639460C98F4
:10C29000F9F738F906460F46099B0E9AF9F780F828
:10C2A000574A0D46914220DB5242AA18024310D150
:10C2B00032463B46F9F718F904900391514A524B24
:10C2C00009990E98F9F76CF8039B049AF9F7DCFAD0
:10C2D0001ED20220FEF72CFBFEF706FB49004908A0
:10C2E000E20FD20711431BB0F0BD6A00474B520862
:10C2F0009A420DD3464AAA18024300D0CBE53246F3
:10C300003B46F9F7F1F8099B0E9AF9F7BDFAF5D912
:10C310006800002340082C490393020D3D4B52183E
:10C32000984223DD01200005521CD04042195000E4
:10C33000400D401838497944096813468C463749FE
:10C34000C1408B4312030121120B0905511814221D
:10C35000101AC1400391002D01DA48420390624651
:10C3600030463946F9F7C0F806460F4632463B4696
:10C3700009990E98F9F714F800252A46284B284603
:10C380000591F9F7BFF807910C90264A264B2846ED
:10C390000599F9F7B7F80091029032463B462846D6
:10C3A0000599F9F7A1F8099B0E9AF9F7A3F81F4A26
:10C3B0001F4BF9F7A7F8009B029AF8F7F1FF074621
:10C3C0000B460246099135E001FCFFFF0000F03FFB
:10C3D0008E9803007AB60B006A070000AC070000D5
:10C3E000D60600000000084009C7EE3FFD033ADC16
:10C3F000F5015B14E02F3EBEAA05000070050000A9
:10C4000000009040FE822B654715973C00CC904081
:10C4100000346F3F0000E03FC6040000FFFF0F0044
:10C42000432EE63F396CA80C615C20BEEF39FAFE62
:10C43000422EE63F07990C98F8F7B2FF05460E46E4
:10C44000079B0C9AF9F750F83A46099BF9F752F80E
:10C4500009912A4633460E9010461946F9F752F8CC
:10C46000074602462F480B46059105217844FEF702
:10C47000CFF93A46059BF9F745F82A463346F9F7CE
:10C4800039F80746019128463146099B0E9AF9F77B
:10C4900039F8099B0E9AF8F783FF012304910C9059
:10C4A00000229B0738460199F9F71EF805910E9076
:10C4B0003A4628463146019BF9F724F8059B0E9A27
:10C4C000F9F788F8049B0C9AF9F70EF82A463346D8
:10C4D000F9F70AF80022144BF9F70CF8064603980E
:10C4E0000D46000541190915002912DC3046294680
:10C4F000039AF9F7E7F8FEF745F9042801D1FEF7AA
:10C50000FDF930462946039AF9F7DCF8064601E0C2
:10C5100004E029180B46324621460898F8F7F2FF46
:10C520001BB0F0BD680300000000F03FF0B58C4682
:10C5300000251026052109078E620E4C08E067468B
:10C540007F5DE760A768FF07FCD0E7681F706D1C80
:10C550008542F4DB0020074606E0E760A568ED07AA
:10C56000FCD0E5681D54401C9042F6D38E6100203B
:10C57000F0BD00000030014070B572B60124074DD7
:10C58000A40221462846F9F757FC002804D0224689
:10C5900003492846F9F7F4FC62B670BD00FC0008B8
:10C5A000DC0D0020F8B506460C46F9F77BFA051EAF
:10C5B0000F4600D00120014349000B484908411AA9
:10C5C000C90F0DD0002E01D0012100E000210C4345
:10C5D00061004908401AC00F02D10120FEF7A8F9F6
:10C5E00028463946F8BD00000000F07FF8B5154632
:10C5F0000E460746002407E03819C0B200F008F8DC
:10C60000641C2870E4B26D1CB442F5D33046F8BD0A
:10C6100010B50446FBF786FFEE20FBF756FFFBF74D
:10C62000BAFF2046FBF751FFFBF7B5FFFBF77AFF98
:10C63000EF20FBF74AFFFBF7AEFF0020FBF718FFE8
:10C640000446FBF78AFF204610BD704770B50D46C3
:10C650000446FBF767FFEE20FBF737FFFBF79BFF76
:10C660002046FBF732FFFBF796FF2846FBF72DFF2E
:10C67000FBF791FFFBF771FF0A20FEF7A2FA70BDEE
:10C68000F0B50025102605279C463F070B46BE62E5
:10C690000C4C06E0595DE160A168C907FCD0E16877
:10C6A0006D1C8542F6DB002007E06146095CE16015
:10C6B000A168C907FCD0E168401C9042F5D3BE6177
:10C6C0000020F0BD0030014000000102030400051D
:10C6D000405C0000A05C0400C06C0800805C0400AA
:10C6E000E03F1E00E07D1E0007A9022570889B88A0
:10C6F0000A001600010006000100020087008D00FC
:10C700002D001A3152001A339A001A351D011A37BA
:10C710006B003B31BE003B335E013B3596023B373D
:10C72000000099599959EB518F421E45142E0080F3
:10C73000EB51F5283333E13A703DE13AC235852BB0
:10C74000C2353333C235C235AE47E13A5138A33032
:10C750005138000000000000000001020304060739
:10C760000809030406080C1018203000000000011E
:10C770000203040000000000000000000000F03F81
:10C78000000000000000F83F000000000000000072
:10C790000000004003B8E23F00000000000000007D
:10C7A00006D0CF43EBFD4C3E033333333333E33F0B
:10C7B000FFAB6FDBB66DDB3F4D268F515555D53F37
:10C7C00001411DA96074D13F65DBC9934A86CD3F05
:10C7D000EF4E454A287ECA3F3E5555555555C53FF3
:10C7E00093BDBE166CC166BF2CDE25AF6A56113FE5
:10C7F000F16BD2C541BDBBBED0A4BE726937663EE7
:10C80000000000000000000028C800080000002010
:10C81000840100006C5B000888C8000884010020C7
:10C820003C1A000020A900080124130704380D0950
:10C830001E080540082609104008560A131D043B2F
:10C8400008BE0516D8BC40100852010336C8420382
:10C85000605C121B0202C5140901022281F01F66EE
:10C8600081049889968696798215980398149887FA
:10C870009674977882439788967197778249D90101
:08C8800045294B9204922000AF
:04000005080050C1DE
:00000001FF
